:100000000266A10269E90000000000026318000016
:10001000000000026A4700000000003200000000FB
:10002000000000022E3D00000000000264440000B9
:1000300000000000000000000000000000000000C0
:100040005052343032207665722E3133322E332EB8
:1000500030204864773A482030352D30312D303605
:100060002030303A3534202075F00612011E22125D
:10007000608F75F00612011E1260942212006F123A
:10008000006812006F12006812006F120068120000
:100090006F12006812006F75F01812011E221260B4
:1000A0008F75F04B12011E12609422754F041227B7
:1000B000A21227B812608F75F0C812011E12609448
:1000C00022754F051227A21227B812009E75F01E46
:1000D00012011E12009E22754F071227A21227B886
:1000E00012008822754F061227A21227B812008E1E
:1000F0002212007C12007C221200E41200E41200A2
:10010000E422C2A1C25012006F75F01212011ED279
:10011000A1C2502212006F75F01212011E22128924
:1001200008201807C0F0128769D0F0D5F0F02270CF
:1001300004A23EB322C0E01412013ED0E022C0E08F
:10014000030303540F28F8D0E0C0E0540704F5F08F
:10015000E213D5F0FCD0E0227003D3802830E7030F
:10016000C3802223F9C3137004A23E801814C0E098
:10017000030303540F2472F8D0E0540704F5F0E2AF
:1001800013D5F0FCE992E022C0E024B0F8E21201BD
:10019000584004D0E0C322D0E024C6F58274003475
:1001A00000F583E01201A82220E702C322C2E7C0C3
:1001B000E0C2E0700AA23EB3D0E030E001B322B466
:1001C0007E03C380F3B40204A22580ECB40404A22D
:1001D0002680E5B40604A22780DEB40804A20380CA
:1001E000D7B40A04A20E80D0B40C0AE56F4570C3E0
:1001F0006001D380C3B40E051262FA80BBB410074D
:10020000A2567255B380B1B41206A255822880A8B6
:10021000B41406A255B028809FB41604A256809844
:10022000B41807740012707A808EB41A0774011221
:10023000707A8084B41C08740212707A0201B8B417
:100240001E08740312707A0201B8B42008740412F4
:10025000707A0201B8B42208740512707A0201B8EB
:10026000B42408740612707A0201B8B42608740720
:1002700012707A0201B8D0E0C3221233F9E5676048
:1002800013B401051202AC8008B402051202C78043
:1002900000756700128769E5715440600B20A8085B
:1002A000304D05C24D1287DF126EC922C23ED26D9B
:1002B000C2AF75186075190F751AFA120BD47577DD
:1002C000031244B3C24022D23EC26DC2AF75187051
:1002D00075190F751AFA120BD475770322C2B6126C
:1002E00069927537007403124BACE51E124BACE5F6
:1002F0001F124BAC7457124BAC120306E537124B6E
:10030000AC3099FDD32278AFE623235403124BACD3
:1003100078B0E630E402240A540F124BAC78AFE612
:10032000C4540375F00AA4F5F0E6540F25F0124BFF
:10033000AC78AEE6C4540375F00AA4F5F0E6540FA9
:1003400025F0124BAC78ADE6C4540775F00AA4F55D
:10035000F0E6540F25F0124BAC78ACE6C4540775A8
:10036000F00AA4F5F0E6540F25F0124BAC78B0E695
:1003700003C45407124BAC2275F032128920B2B577
:10038000128920B2B5D5F0F322D2A3C24ED2A2C2B6
:1003900051C2A1C250D2A4C24FC2A012608F120398
:1003A00078D2A0126094120378C2A012608F120358
:1003B00078D2A0126094120378C2A012608F120348
:1003C00078D2A01260941203781203781203781284
:1003D000037812037822E9C4540F2323F890052AE6
:1003E00093FF08E893FE08E893FD08E893FCE954BE
:1003F0000F601BF82328F89004FA932FD4FF08E825
:10040000933ED4FE08E8933DD4FDE43CD4FCEA607E
:100410003CC4540F601BF82328F89004CD932FD4CC
:10042000FF08E8933ED4FE08E8933DD4FDE43CD4B5
:10043000FCEA540F601723F89004B0932FD4FF0800
:10044000E8933ED4FEE43DD4FDE43CD4FCEB6034C0
:10045000C4540F601723F8900492932FD4FF08E838
:10046000933ED4FEE43DD4FDE43CD4FCEB540F6059
:1004700013900484932FD4FFE43ED4FEE43DD4FDD6
:10048000E43CD4FC2201020304050607080910110C
:100490001213141516003200480064008000960004
:1004A0001201280144016001760192010802240230
:1004B0004002560212056807241080123615921762
:1004C00048200423602516287230283384354038AC
:1004D00096400092810088220184630180040276A4
:1004E0004502728602682703646803600904565057
:1004F00004529104483205447305401406365506EB
:100500007210130866194421268076321632395249
:100510008745884252249858605365960872326421
:100520007868198504759140309800000000768540
:100530000401527109022857140304431904802846
:1005400024055614290632003407088638088471B9
:100550004309605748103643531112295812881422
:1005600063136400681440867215C0F075F0DCD522
:10057000F005B2B5120738C0F012072BD0F030E703
:10058000EED0F022AAF012056AE532652FF5F0E50B
:1005900033653045F0600C12067A852F3285303392
:1005A00012056A1206F012056A12071812056A127D
:1005B00006878AF022AAF012056AE532652FF5F067
:1005C000E533653045F0600C12067A852F328530B0
:1005D0003312056A1206DC12056A12071812056A40
:1005E0001206878AF022AAF012056AE532652FF515
:1005F000F0E533653045F0600C12067A852F3285C0
:10060000303312056A1206AC8AF022AAF012056A8B
:10061000E532652FF5F0E533653045F0600C1206E4
:100620007A852F3285303312056A1206948AF022B9
:10063000C0F075F00833C297928300D297D5F0F5D9
:10064000D0F022C0F075F008C297D29700A2823392
:10065000D5F0F5D0F022D2B7D297D283D282D2840D
:1006600022120630E53033E52F33120630C3E53071
:1006700033120630E53112063022120656C2847457
:1006800053120661D28422120656C284745812068E
:1006900061D28422120656C2847454120661E41296
:1006A0000630120643F608D9F9D28422120656C241
:1006B000847454120661E4120630120643F208D91B
:1006C000F9D28422120656C2847454120661E412CE
:1006D0000630120643F0A3D9F9D28422120656C27C
:1006E000847484120661E612063008D9F9D2842295
:1006F000120656C2847484120661E212063008D9CA
:10070000F9D28422120656C2847484120661E01261
:100710000630A3D9F9D28422120656C284748312F9
:100720000661D28412890812890822C28474571281
:100730000630120643D2842275F06412072B20E59E
:100740000430E30122C2AFB2B5128920B2B51289DA
:1007500020D5F0E712038980FBD283D282D297D2D0
:10076000B7D284B2B575F002128908D5F0FAC2B7D3
:10077000B2B575F002128908D5F0FAD2B7B2B52237
:100780007920752F017530037531E09000DC12057A
:100790006A12067A12056A1206C47900752F01756D
:1007A00030047531009000FC12056A12067A1205B9
:1007B0006A1206C479E0752F017530057531009015
:1007C00001FC12056A12067A12056A1206C4852F08
:1007D0003285303322752F017530DB7531001205FB
:1007E0006A120A707532FF7533FF22AE83AD8290B4
:1007F000DB007F207404F974AAF8752F018583301B
:1008000085823112060B78AAE66E702508E66D70B7
:100810002008E6601AB4FF028013167404F974AA63
:10082000F8752F018583308582311205B5C322D337
:1008300022A3A3A3A3DFBD80F490DB007F20740478
:10084000F974AAF8752F0185833085823112060B61
:1008500078AAE66E700908E66D700408E6FC22A32B
:10086000A3A3A3DF0A7CFF2290DB007F207BFF7421
:1008700004F974AAF8752F01858330858231120638
:100880000B78AAE66E702C08E66D702708ECB4FFB2
:100890000D78AA76FF0876FF0876FF0874FFF674D5
:1008A00004F974AAF8752F01858330858231120509
:1008B000B5C322BBFF1078AAE6B4FF0A08E6B4FF6E
:1008C00005C374209FFBA3A3A3A3DFA3BBFF02D395
:1008D00022EB232354FC2400F5827583DB500205B0
:1008E0008378AAEEF608EDF608ECF608E4F6740450
:1008F000F974AAF8752F018583308582311205B508
:10090000C32275830075F08E752F02858330753193
:1009100000C0F0C08312056A120A70D0830583D02C
:10092000F0D5F0E475830075F0DA752F0385833018
:10093000753100C0F0C08312056A120A70D08305B9
:1009400083D0F0D5F0E47532FF7533FF2275830054
:1009500075820075F08EC0F0C082C083752F02854D
:10096000833075310012056A12067AD083D082C0B6
:1009700082C083752F0085823075310012056A129E
:100980000718D083D08205830582D0F0D5F0C775D3
:10099000830075820075F0DAC0F0C082C083752FC5
:1009A0000385833075310012056A12067AD083D030
:1009B00082C082C083752F01858230753100120597
:1009C0006A120718D083D08205830582D0F0D5F053
:1009D000C77532FF7533FF2275830075820075F08D
:1009E0008EC0F0C082C083752F00858330753100C2
:1009F00012056A12067AD083D082C082C083752F16
:100A00000285823075310012056A120718D083D032
:100A10008205830582D0F0D5F0C77583007582000A
:100A200075F0DAC0F0C082C083752F018583307500
:100A3000310012056A12067AD083D082C082C08348
:100A4000752F0385823075310012056A120718D0A0
:100A500083D08205830582D0F0D5F0C77532FF754B
:100A600033FF22120656C2847450120661D28422C9
:100A7000120656C2847481120661D284221206566E
:100A8000C2847484120661E8120630D9FAD2842234
:100A9000F8790012056A120A7DEAC0E085822F8586
:100AA000833075310012056A120718D0E0FA058309
:100AB000DAE77532FF7533FF22120656C28474548A
:100AC000120661E4120630E4C0E0120643D0F025BD
:100AD000F0D9F5D284227583007582028006758371
:100AE00000758200E475F08D85822F858330753125
:100AF00000C082C083C0F0C0E012056A12067A12FC
:100B0000056A7900120AB9D0F025F0D0F0D083D070
:100B1000820583D5F0D285822F858330753100C060
:100B2000E012056A12067A12056A7920120AB9D013
:100B3000F025F07532FF7533FF227583007582034F
:100B40008006758300758201E475F0DA85822F8551
:100B50008330753100C082C083C0F0C0E012056AE6
:100B600012067A12056A7900120AB9D0F025F0D07F
:100B7000F0D083D0820583D5F0D27532FF7533FF74
:100B800005E02275830075F000752F0085833075B0
:100B90003100C0F0C08312056A120A70D083058349
:100BA000D0F0D5F0E47532FF7533FF75830075F032
:100BB000DA752F01858330753100C0F0C0831205CE
:100BC0006A120A70D0830583D0F0D5F0E47532FF45
:100BD0007533FF2253550F53540F5318F053190F09
:100BE000C2AFE55423247CF8E5184519F608A61A87
:100BF000055453540FE554B55505055553550FD2BB
:100C0000AFC3E55495555002241024F45003755F8A
:100C10000022E555B554057400780022C333247CC6
:100C2000F8E6C0E008E6F8D0E02253540F53550F21
:100C3000C2AFE555B55404D2AFD322055553550F75
:100C4000D2AFC322300C2D78AFE6540FC0E0E6C41B
:100C5000540375F00AA4D0F025F0FD78B0E630E436
:100C600002240A540FFE901A00120C75400690D30D
:100C700000120C75227F3C7404F97400F8752F0182
:100C80008583308582311205E67800E26D701708A1
:100C9000E26E701208E2C42354E0F5F078B0E65436
:100CA0001F45F0F6D322A3A3A3A3DFCBC32212696F
:100CB00092120C441269A1FEAFF07DFF0DED30E7FA
:100CC0000122D25975F004A424DCF582E5F0340049
:100CD000F583C082C08378AAE0F6A308E0F6A308F3
:100CE000E0F6A308E0F6D083D08278AA868308864F
:100CF0008278AAB6FF0708B6FF03020D74C3E58227
:100D000033F582E58333F583E58224E0F582E583DC
:100D10003405F58378ACE6705B08E66057FB740237
:100D2000F974AAF8752F0185833085823112060B7C
:100D3000A3A378AAE60856B4FF03020D7478AA8626
:100D4000F053F07F08E6C39EC5F09F401E7025E576
:100D5000F06018BD001E203E1B78AAE6A2E720E73F
:100D600013E5F024FA400DD268800978AAE6A2E7DC
:100D70009259DBAABD00028028ED14C0E0030303F2
:100D8000540F2472F8D0E0540704FB7400D333DB13
:100D9000FD305905FBE24B8004F4FBE25BF2020CF0
:100DA000BCB2591287B8406F202F6C206C69201993
:100DB0000B203D05305960800320595B30593D20A0
:100DC0003D3A78AFE2702F20672178ADE2602D12B6
:100DD000665B6028F5F0E5F0543F4400C2AF75183B
:100DE000C0751909F51A120BD4800512665B600CE8
:100DF00078ADE278AFF2D268D267801BC268C26772
:100E0000A259923D400B303E0E120E1A1243FB8047
:100E100006203E03120E35020CBCC23ED26DC2AF9C
:100E200075186075190F751AE0120BD475770312D7
:100E300044B3C24022D23EC26DC2AF75187075195C
:100E40000F751AE0120BD475770322120630E530C5
:100E500033E52F33120630C3E53033D2E0120630CB
:100E6000E53112063022120656C2847454120E4B1B
:100E7000E4120630120643F608D9F9D2842212068B
:100E800056C2847484120E4BE612063008D9F9D289
:100E9000842290FC00752F04753000753100C082EB
:100EA000C0837549FA12056A12067A852F66853065
:100EB00065790878AA12056A120E661210E6D083C8
:100EC000D0827044C082C08378AE86830886821246
:100ED0000F3F402478AC8683088682120F3F40186B
:100EE000120F5EE582600AE563B5650CE564B566E0
:100EF00007D083D082020F1A78ACE6249AF612113A
:100F000029120389D083D0820530E5307002052F85
:100F1000A3E58245837087120F217532FF7533FF79
:100F20002278AC760008760078AE76000876000865
:100F3000760008760075660475650012110522C0FA
:100F400082C083E5822400F582E5833480F5834006
:100F500005D083D08222D083D08290000022E58207
:100F600075F008A4F582E5F0C58375F008A4258323
:100F7000F583E5F03404F564E5822400F582E58329
:100F80003400F5835002056485836322120389D0FF
:100F900083D08222C082C0831210BF70EF78AC86EB
:100FA00083088682120F3F40E3120F5E1213A0786F
:100FB000AA760078AEE518F608E519F60876000876
:100FC00076007408F974AAF885642F8583308582C9
:100FD000311205B57404F974AEF885642F85833039
:100FE00085823112060B75F00478AA79AEE6676047
:100FF0000280990809D5F0F51210C678AC868308EE
:101000008682A3120F3F78ACA68308A68278AE86AC
:1010100083088682120F3F78ACE66583706208E62B
:101020006582705CC064C063C082C083120F5E744E
:1010300008F974B2F885642F8583308582311206F1
:101040000B78B676C0087657087600087600D0830D
:10105000D082E582241EF58250020583120F3FC024
:1010600082C083120F5E7408F974B2F885642F850C
:1010700083308582311205B5D083D082D063D064AD
:1010800078AEA68308A682C066C06585646685635F
:1010900065121105D0E0D0F0B56509C5F0B566025E
:1010A0008018C5F0C066C06585F066F56578ACE669
:1010B0002499F6121129D065D066D083D0822212ED
:1010C00010C61210E62285662F8565307531001234
:1010D000056A12067A790878AA12056A120E6685E0
:1010E0002F328530332278AFE618261826182618B6
:1010F000245566700F78AFE618661866186618668D
:10110000186499662212110C1211292278AFE61880
:101110002618261826182455F678AFE6186618669D
:1011200018661866186499F62285662F85653075ED
:10113000310012056A12067A12056A790878AA1235
:101140000E7E12056A12071812056A120687852F8D
:1011500032853033221210BF703078ACE6C0E00820
:10116000E6C0E0088683088682C3D0E09582F582D7
:10117000D0E09583F58350104582600CE582240011
:10118000F582E5833480F583C322900000D322C228
:10119000B6121155E433C0E07537007403124BAC3E
:1011A000E51E124BACE51F124BAC7453124BACD086
:1011B000E0124BAC7400124BAC7400124BACE583E4
:1011C000124BACE582124BACE537124BAC3099FDBB
:1011D00022C2B6E5356004F4FF8004FF120F2175CA
:1011E00037007403124BACE51E124BACE51F124BDB
:1011F000AC7456124BACEF124BACE537124BAC3023
:1012000099FD227401C0E078AA75F008E4F608D5CB
:10121000F0FBD0E0D32212115540E860E878AE86AA
:1012200083088682121229C322C082C083E5827598
:10123000F008A4F582E5F0C58375F008A42583F5D0
:1012400083E5F03404F564E5822400F582E5833417
:1012500000F583500205647408F974AAF885642FB8
:1012600085833085823112060BD083D08222121101
:10127000557F085005120F217F0078AC86560886EE
:1012800057088658088659C2B67537007403124B42
:10129000ACE51E124BACE51F124BAC7454124BACB8
:1012A000E535124BACEF124BACE535603CE55965CA
:1012B00057F5F0E558655645F0600B85598285581D
:1012C000831212298003121205855982855883A33F
:1012D000120F3F85825985835878AA75F008E61267
:1012E0004BAC08D5F0F8D535C4E537124BAC309986
:1012F000FDC322E5357007C2AF1211555005E53523
:10130000F4800C78AEA65808A659121105E535D21E
:10131000AFC0E0C2B67537007403124BACE51E12C5
:101320004BACE51F124BAC7455124BACD0E0124BDA
:10133000ACE537124BAC3099FDD322C2B6753700FD
:101340007403124BACE51E124BACE51F124BAC7490
:1013500058124BAC7420232354FC04124BAC742061
:10136000124BAC90DB007F207404F974AAF8752F3F
:101370000185833085823112060B78AAE6124BACC8
:1013800008E6124BAC08E6124BAC08E6124BAC0870
:10139000A3A3A3A3DFD2E537124BAC3099FDD32230
:1013A00012699278B0E630E402240A540FC4F97846
:1013B000AFE6C4540375F00AA4F5F0E6540F25F027
:1013C000C3134978ABF678AFE692E754C0F978AD2D
:1013D000E6C4540775F00AA4F5F0E6540F25F04969
:1013E000F978AEE6C4540375F00AA4F5F0E6540F9C
:1013F00025F0F5F078ACE654702345F078ADF6783A
:10140000ACE9F62222303FFD12608F75F006120122
:101410001E12609475F01412011EE53FC23F22E4D3
:101420002278AA7910E6B5F0070805F0D9F7E4228A
:10143000740122C0E078AA7910F60805E0D9FA74A0
:1014400010F974AAF8752F037530DB753100120599
:10145000B57410F974AAF8752F037530DC75310076
:101460001205B57410F974AAF8752F037530DB7581
:10147000310012060BD0F0C0F0121421701E74104F
:10148000F974AAF8752F037530DC75310012060B5C
:10149000D0F0C0F01214217003D0F022D0F022E579
:1014A0001DC0E0121433D0F07006E5F0F4121433CE
:1014B00022785074FFF21215E8C20C120B42600140
:1014C000221207807401F97450F8752F01753003EA
:1014D0007531A01205E67410F97482F8752F017544
:1014E00030037531C01205E67410F97492F8752F47
:1014F000017530037531D01205E67402F9745FF896
:10150000752F017530CE7531001205E67416F97429
:10151000B0F8752F017530CE7531C01205E678B080
:101520009000C675F016E2F008A3D5F0F97416F92C
:1015300074B0F8752F017530037531A11205E6748A
:1015400008F97400F8752F017530D2753100120555
:10155000E678009002EF75F008E2F008A3D5F0F904
:101560009002F4E0B4FF14A3E0B4FF0FA3E0B4FFD3
:101570000A9002F47483F0A3F0A3F0D20CE4227971
:10158000AA776509E4A23E92E0A23D92E7F70974CA
:1015900004F974AAF8752F0275308E7531001205A2
:1015A000B522D23EC26DD23D22C26C7404F974AA37
:1015B000F8752F0275308E75310012060B78AAB6B9
:1015C00065E008E6D26CA2E0923EB3926DA2E7928B
:1015D0003D78AA76FF7401F974AAF8752F02753068
:1015E0008E7531001205B52278B075F016E4F20858
:1015F000D5F0FB74FF78B8F278B9F2227403F9746D
:101600005AF8752F0075308C7531E51205E6785A59
:10161000E224FD9208E224E292097401F97459F877
:10162000752F0075308C7531E21205E67859E22489
:10163000FD9206E224E29207227403F9745AF875C7
:101640002F0075308C7531E51205847401F97459D9
:10165000F8752F0075308C7531E21205842279AA55
:10166000774809774E0977840977A07404F974AA3A
:10167000F8752F0075308D7531201205B57404F999
:1016800074AAF8752F0275308D7531201205B522B8
:101690007404F974AAF8752F0075308D7531201215
:1016A000060B79ACE7648422E4A21E92E0A21F92AA
:1016B000E1A22092E2A20192E379AAF77401F974FF
:1016C000AAF8752F0075308C7531E81205B52274B3
:1016D00001F974AAF8752F0075308C7531E812067F
:1016E0000B79AAE7A2E0921EA2E1921FA2E2922049
:1016F000A2E392012279AAE4A22B92E0A22C92E129
:10170000A22D92E2A21692E392E492E5A22F92E633
:1017100092E7F709E4A22E92E0A23092E1A2319280
:10172000E2A23292E3A23492E6A23592E7F709E40C
:10173000A23692E0A23892E2A23992E3A23A92E46F
:10174000A23B92E5A23C92E7F709E571F77404F930
:1017500074AAF8752F0075308C7531EC1205B579C7
:10176000AAE572F4F709E573F4F709E574F4F77480
:1017700003F974AAF8752F0075308C7531E91205DC
:10178000B5227404F974AAF8752F0075308C753180
:10179000EC12060B79AAE7A2E0922BA2E1922CA20E
:1017A000E2922DA2E39216A2E6922FA2E709E7A207
:1017B000E0922EA2E19230A2E29231A2E39232A212
:1017C000E69234A2E7923509E7A2E09236A2E292CD
:1017D00038A2E39239A2E4923AA2E5923BA2E6A2B1
:1017E000E7923C09E7F5717403F974AAF8752F00C4
:1017F00075308C7531E912060B79AAE7F4F5720998
:10180000E7F4F57309E7F4F5742279AAF77401F99E
:1018100074AAF8752F0075308C7531E41205B52265
:101820007401F974AAF8752F0075308C7531E412C3
:10183000060B79AAE7227401F9744AF8752F00752E
:10184000308C7531FC120584227401F9744AF875E4
:101850002F0075308C7531FC1205E622784AE27053
:1018600006784BF208F22275F000303A0475F03C2D
:10187000A4AAF075F008A4FBACF0EA75F008A42C5B
:10188000FAC374FD9BFB74FF9A784BF2EB08F222CB
:101890007401F9744DF8752F0075308D7531001293
:1018A0000584227401F9744DF8752F0075308D751B
:1018B00031001205E6227402F97468F8752F00757C
:1018C000308C7531FD1205E67402F9746AF8752FD3
:1018D0000075308D7531011205E6227402F97468C5
:1018E000F8752F0075308C7531FD1205847402F97E
:1018F000746AF8752F0075308D75310112058422D8
:101900007401F97451F8752F0075308C7531F0122F
:1019100005847401F97452F8752F0075308C753197
:10192000F41205847401F97453F8752F0075308C26
:101930007531F61205847401F97454F8752F007529
:10194000308C7531F2120584227401F97451F875E6
:101950002F0075308C7531F01205E67401F9745260
:10196000F8752F0075308C7531F41205E67401F9A5
:101970007453F8752F0075308C7531F61205E674C6
:1019800001F97454F8752F0075308C7531F2120519
:10199000E6227401F97438F8752F0075308C7531B2
:1019A000F81205B57401F97439F8752F0075308C8B
:1019B0007531FA1205B57401F9743AF8752F00758E
:1019C000308C7531FB1205B5227401F97438F87545
:1019D0002F0075308C7531F812060B7401F97439CB
:1019E000F8752F0075308C7531FA12060B7401F9F9
:1019F000743AF8752F0075308C7531FB12060B2286
:101A00007402F9741EF8752F0075308C7531E01270
:101A100005B5227402F9741EF8752F0075308C75A7
:101A200031E012060B22E57454026003756A1878DF
:101A3000C379AEE56A800075F00484FAC0F08002D4
:101A40001819E7F5F066540F7036DA0CD0E0602E06
:101A5000FA18E7C4F5F0801618E7C4F5F066540FDD
:101A6000701EDADCD0E06016FA1819E7F5F0E4D35E
:101A700033DAFCFAE65AC5F05AC395F0700EE42248
:101A8000D0E0E6540FC5F0540FC395F0920B7401EB
:101A90002278AF79217A03E6C4540FF309E6540F94
:101AA000F30908DAF2792178C67A06E6540FF6E3EC
:101AB0006670080908DAF4E4C24122792678CB7A04
:101AC00006C3E3961918DAFA920B792678CB7A06D0
:101AD000E3540FB40F08E6540FB40F108008E65417
:101AE0000FB40F0B80061819DAE680CB740122C3FD
:101AF000E396B40902801214600FC3E3F5F0E69593
:101B0000F0B4090280031470E3E9B42104E4D24183
:101B1000221918E366540F60F080D178AF79C67A45
:101B200003E7540FC4F5F009E7540F45F086F0B50C
:101B3000F0060908DAEBE422B3920B740122121AC0
:101B400091701F30411C202E1AC2AF75185085832A
:101B50001985821A120BD47575007405127031D272
:101B600040E42204227408F974AAF8752F00753035
:101B70008C7531C012060B121A26227408F974AA49
:101B8000F8752F0075308C7531C012060B121B3E94
:101B9000227405F974AAF8752F0075308C7531C060
:101BA0001205B5227403F974AFF8752F0075308CE7
:101BB0007531C51205B522C082C083E5822420F5A7
:101BC00082E583347DF5837401F9743BF8752F0049
:101BD00085833085823112060BD083D082C082C0CB
:101BE00083E58275F008A42420F582500205F0A850
:101BF000F0E58375F008A4282400F5837408F974CF
:101C0000AAF8752F0085833085823112060BD083A8
:101C1000D082123F3522C082C083E58275F008A4CD
:101C20002420F582500205F0A8F0E58375F008A4A1
:101C3000282400F5837408F974BAF8752F00858399
:101C40003085823112060BD083D08222C082C083BD
:101C5000E58275F008A42420F582500205F0A8F072
:101C6000E58375F008A4282400F5837406F974AAA6
:101C7000F8752F0085833085823112060BD083D012
:101C800082227405F974AAF8752F00753000753139
:101C90002012060B121A2622900000121BB7121AED
:101CA0002622300CF3751B00751C0075619F756250
:101CB0000FE561251BC2E0F582E562351CF583C0A6
:101CC00082C083E5822400F582E583341BF58374AA
:101CD00002F974AAF8752F018583308582311206C6
:101CE0000B78AA8683088682121BB7121A26700503
:101CF000D0F0D0F022D083D082C3E58313F583E502
:101D00008213F582200B14E58245836022E582244C
:101D1000FFF561E58334FFF5628007A385821B85AB
:101D2000831CC3E561951BE562951C4002808274AB
:101D30000122300C397410F974AAF8752F0175302E
:101D4000CE75312012060B78BA79AA75F00AE7B47D
:101D5000FF02801AB43C120809D5F0F2900FE8781F
:101D6000BEE2F53B784FF2E42266540F60E974015D
:101D700022900000121BB7121B3E2278C6E6540FB9
:101D8000B40F03021E15200C0280E6751B00751CA3
:101D90000075619F75620FE561251BC2E0F582E564
:101DA00062351CF583C082C083E5822400F582E59C
:101DB00083343BF5837402F974AAF8752F01858387
:101DC0003085823112060B78AA8683088682121B20
:101DD000B7121B3E7005D0F0D0F022D083D082C362
:101DE000E58313F583E58213F582200B14E5824524
:101DF000836022E58224FFF561E58334FFF562808C
:101E000007A385821B85831CC3E561951BE562954D
:101E10001C4002808274012230470DE536B443082D
:101E2000E53424FE500280F078BA7A0579CEE65483
:101E30000FC4F5F008E6540F45F0F70809DAEF2271
:101E400075F01E128908D5F0FA1200E475F00F1231
:101E50008908D5F0FA1200E475F00F128908D5F060
:101E6000FA1200E422120094B2B575F00F1289083C
:101E7000D5F0FA30B7EF22D218D2A3C24EC2A2D206
:101E800051D2A1C250D2A4C24F121E65121E4012DE
:101E900021311258EE12692E120F211207D5C2A35A
:101EA000C24EC2A2C251C2A1C250D2A4C24F12603D
:101EB000B94005C2AF026613120094B2B575F00FB7
:101EC000128908D5F0FA80E6C2A3C24EC2A2C2515E
:101ED000C2A1C250D2B775F002128908D5F0FA201B
:101EE000B7441260B95002808ED218D2A3C24EC23B
:101EF000A2D251D2A1C250D2A4C24F121E65D21892
:101F0000125934401CC2A3C24EC2A2C251C2A1C2C5
:101F100050D2A4C24F12205A1258EE120F211207AB
:101F2000D5C2AF026613126094C01D120ADED0F053
:101F3000703BC3E51D95F078A4F2121FF4121690C1
:101F40006019D218900000121BB712205A1258EED6
:101F5000120F211207D5B2B5121FF41214B1E57495
:101F60005408700812690B5003121FAF22D2A3C28B
:101F70004ED2A2C251C2A1C250D2A4C24FC2187541
:101F800049FAC2A075F0C8128908D5F0FA12608F1C
:101F9000D2A075F0C8128908D5F0FA1260941234F4
:101FA00082D2B712892020B7C4021EE2020000D2FA
:101FB000B712892030B7F5D2A3C24ED2A2C251C205
:101FC000A1C250D2A4C24FC2187549FAC2A075F07E
:101FD00014128908D5F0FA12608FD2A075F014128D
:101FE0008908D5F0FA126094125B99123482126952
:101FF0000B40BC221216CF121782121820A2E492B4
:102000006FA2E59270A2E69271A2E792721218494D
:102010001218A31219491219C91218B67401F974C9
:10202000ADF8752F017530CE7531301205E678ADFB
:10203000E2B4FF02E4F27401F974AEF8752F017591
:1020400030CE7531311205E678AEE2B4FF02E4F22B
:10205000121A131215FC12185C22D218C2A3C24E17
:10206000C2A2C251C2A1C250D2A4C24FC01EC01F40
:1020700078AA9000007A08E6F008A3DAFA12213173
:1020800012692E78AA9000007A08E0F608A3DAFA1E
:1020900090000012585D121B91121BA4D01FD01E7D
:1020A000121A0022751E30751F30D21EC21FC220A8
:1020B000C201C22BC22CC22DC216C22FC22ED230D8
:1020C000C231C232C234C235C236C238C239C23A53
:1020D000C23BC23C7571007572007573007574085F
:1020E00078687422F2087400F2786A7406F2087450
:1020F00000F2C26FC270C271C272784A7404F27880
:102100004D7409F278517401F278527402F27853E6
:102110007404F278547404F2753807753900753A0E
:102120000074017859F2785AF2E408F208F2C20C0D
:1021300022120B831220A4121A001216A81216F5EE
:10214000C2E0A26F92E4A27092E5A27192E6A2723E
:1021500092E712180A121836121890121900121962
:10216000921218DB12163912165E126113223053C6
:1021700004C253800975F00C20B205D5F0FAD322C1
:10218000C322E8C0E0E9C0E0EAC0E020063720084A
:102190003412216E5025754F00785AE2600C75F0AC
:1021A00003128908D5F0FA1224B37859E2600C754D
:1021B000F003128908D5F0FA122624D0E0FAD0E014
:1021C000F9D0E0F822200916200713305DEDC08217
:1021D000C0831221F5126A85D083D08280DD305D04
:1021E000DAC082C083E5697003122253126BE3D018
:1021F00083D08280C630050C300609D258C2577889
:102200005902220D3008F4D257C258785AE2B40F5E
:1022100002801BB410071240B8D2498035B41105B2
:10222000123FC9802075F00384E5F0B40007124125
:1022300043D249801DB40107124061D2488013B4D3
:102240000210123FED400B7848E583F208E582F278
:10225000D24A2230050C300709D258C257785902A9
:10226000226B3009F4D257C258785AE275F00384D1
:10227000E5F0B400091242E94020D249801CB401C3
:10228000091243114014D2488010124314400B78B5
:1022900048E583F208E582F2D24A22D24B8008C296
:1022A0004B12230D753C00C217D2537549FA744086
:1022B000301802740CF547C249C23FE54760391235
:1022C000218220493375F003128908D5F0FA1202F1
:1022D0007A201803201718303FE1204B1B75476008
:1022E000121405B40B0D75F008128908D5F0FAD256
:1022F00049800512230080C3C248D2AF7549FA2233
:10230000533C07F8E53C24C6C8F6053C2278C67560
:10231000F00874FFF608D5F0FB22304809201D03B1
:10232000D21D22C24822C21D22D24B8009C24B7448
:102330001002233DC24B7440301802740CF547D292
:1023400053C217D21C7549FA12230D753C00C249BD
:10235000C248C23FC24AC24C12027A201803201758
:102360002D122182204929204826204A23303F2D42
:102370007859E27004C23F8024204B1475476012E4
:102380001405B40B1275F008128908D5F0FAD24979
:102390007575037549FA22757503122300E54760C8
:1023A000F2304CFD80B0B40207204907C248C24A4F
:1023B000022434C082C08390EA60E53C606324FB61
:1023C000405F78C6E6540F758300F582D53C0280E5
:1023D0005075F00AA4F58275830008E6540F258233
:1023E000F582D53C02803AE58275F00AA4F5828533
:1023F000F08308E62582F58250020583D53C0280F1
:1024000020E58275F00AA4F582C0F0E58375F00A34
:10241000A4D0F025F0F58308E62582F58250020568
:10242000837848E583F208E582F2C249C248D24A7D
:10243000D083D08222C289C28BD293C2B422C0F090
:1024400075F0FAD5F0FD75F064D5F0FDD0F02212EC
:10245000243E12243E12243E12243E12243E122414
:102460003E22D293C2B475F00512892020B2061222
:10247000892030B203D5F0F112892022C0F075F026
:1024800008A2E7B392B4C29312243EC2B4D293120C
:10249000243EC0E0E430B201040030B20104003058
:1024A000B20104D36003D5E001C3D0E033D5F0D14D
:1024B000D0F022D293C2B4D2B212243EC2931224DC
:1024C0004FD29312244F20181F30582378A2760140
:1024D000087480F608A2A3B392E4F6749008F60894
:1024E000F608F608F602252C78A276050224F37881
:1024F000A27603087680087480A24E92E5A2A3B368
:1025000092E4201808A25192E1A22892E0F6087401
:102510008020580FE54F54074480A25092E5A2A1B5
:10252000B392E4F6087480F608F608F675F00778BA
:10253000A27E007F00E62EFEE612247CF62FFF0826
:10254000D5F0F2EED33312247CF8EFD33368706405
:1025500078A2B6FF5F055DE55D24FE5016755D024D
:10256000201A10D21AC2AF7518C0751900751A0357
:10257000120BD4785AE2600330580302262078A860
:10258000E620E36620E25620E14978A3E6B6002281
:1025900008B6420A08E6D257122A7E022620B6550D
:1025A0001108B6000D087948E6F30809E6F3D24AA7
:1025B000D257806CE55D6019D55D16301A13C21ACA
:1025C000C2AF7518C0751900751A04120BD4757650
:1025D00003804DD25778A3863FD23F804378A386AD
:1025E0003C08D24979C67A04800B78A3D248756A30
:1025F0002879BA7A05D25775F00FE6C4540FF7550B
:10260000F0F5F009E6540FF755F0F5F00908DAEAAD
:10261000E5F0B40F051977EEC248785AE21223A606
:1026200012246222D293C2B4D2B212243EC29312B6
:10263000244FD29312244F20181F30572378A276AC
:1026400011087480F608A2A3B392E4F6749008F619
:1026500008F608F608F60226A978A276150226647E
:1026600078A27613087680087480A24E92E5A2A321
:10267000B392E4205714A24F92E1A2A4B392E020B7
:102680001808A25192E1A22892E0F608748020571F
:102690000FE54F54074480A25092E5A2A1B392E403
:1026A000F6087480F608F608F675F00778A27E0042
:1026B0007F00E62EFEE612247CF62FFF08D5F0F20E
:1026C000EED33312247CF8EFD33368706478A2B66B
:1026D000FF5F055CE55C24FE5016755C02201B1054
:1026E000D21BC2AF7518C0751900751A05120BD42C
:1026F0007859E2600330570302279E78A8E620E36A
:102700006720E25720E14A78A3E6B6002208B642E5
:102710000A08E6D258122A7E02279EB6551108B63C
:10272000000D087948E6F30809E6F3D24AD258804A
:102730006DE55C6019D55C16301B13C21BC2AF750A
:1027400018C0751900751A06120BD4757603022786
:102750009ED25878A3863FD23F804378A3863C0818
:10276000D24979C67A04800B78A3D248756A287951
:10277000BA7A05D25875F00FE6C4540FF755F0F544
:10278000F009E6540FF755F0F5F00908DAEAE5F03C
:10279000B40F051977EEC2487859E21223A6122425
:1027A0006222785AE2601024FD400C75F003128911
:1027B00008D5F0FA1224B3227859E2601024FD40C3
:1027C0000C75F003128908D5F0FA12262422C0E015
:1027D00030570EC2AF7518B0751900751A00120B7C
:1027E000D4D0E022D293C2B4D2B212243EC2931209
:1027F000244FD29312244F78A2E56D540FC444079E
:10280000F608E56C23A2E392E5A2E292E3542AD211
:10281000E7F608E56CA2E392E1A2E492E3542AD23F
:10282000E7F608E56CA2E692E1A2E792E3540AD249
:10283000E7F6748008F608F608F675F00778A27EC9
:10284000007F00E62EFEE612247CF62FFF08D5F06E
:10285000F2EED33312247CF8EFD33368700B78A2F6
:10286000B6FF06122462C38004122462D322756D5F
:1028700008786CE2F56C1227E474004005122948D0
:102880008003122970756D09786DE2F56C1227E4EA
:102890007401400512294880031229702222E57133
:1028A000542060F9756D04756CFF1227E4740250B2
:1028B000041229702212294878A57943E6F3080901
:1028C000E6F3087945E6F30809E6F378A3E6A2E023
:1028D00092E25414F5F008E623A2E592E054034591
:1028E000F0F5F07847E265F0C0E0E5F0F2D0E030D6
:1028F000E221C0E0C0F0E5F075F04930E20375F088
:102900004AC2AF7518C075190085F01A120BD4D0E1
:10291000F0D0E054037003022947E5F05403B403F8
:102920000575F0488013B4020575F047800BB400BC
:102930000575F04B800375F04CC2AF7518C0751962
:102940000085F01A120BD422F5F0242AF8E2B40222
:1029500005227402F22250FA7402F2E5F02432F5F4
:10296000F0C2AF7518C075190085F01A120BD42289
:10297000F5F0242AF8E2601CD5E018F2E5F0243CDA
:10298000F5F0C2AF7518C075190085F01A120BD496
:10299000757603F222D293C2B4D2B212243EC2930D
:1029A00012244FD29312244F78A2E56D540FC444E1
:1029B00003F6087680087480A24E92E5A2A3B39233
:1029C000E4A25192E1A22892E0F6087480A250920B
:1029D000E5A2A1B392E4F6087480F608F608F6754D
:1029E000F00778A27E007F00E62EFEE612247CF639
:1029F0002FFF08D5F0F2EED33312247CF8EFD33357
:102A000068707178A2B6FF6C78A8E620E33020E207
:102A10002020E16078A3E6B6005A08B6551108B642
:102A20000052087948E6F30809E6F3D24A804A8062
:102A30004378A3863C08D24979C67A04800B78A3F0
:102A4000D248756A2879BA7A0575F00FE6C4540F32
:102A5000F755F0F5F009E6540FF755F0F5F00908D1
:102A6000DAEAE5F0B40F051977EEC248785DE212B4
:102A700023A68005122462D322122462C322B4FF4B
:102A800017D2647568051227CEC2AF7518C07519C4
:102A900000751A07120BD422B4BC03022AB1B4BDCC
:102AA00003022AE3B4BE03022B15B4BF03022B4773
:102AB000222057147408F974AAF8752F017530CEC6
:102AC00075314012060B80127408F974AAF8752F3C
:102AD000017530CE75314812060B741178B2F612BA
:102AE0002B79222057147408F974AAF8752F0175F0
:102AF00030CE75315012060B80127408F974AAF8A2
:102B0000752F017530CE75315812060B741278B2DC
:102B1000F6122B79222057147408F974AAF8752F2D
:102B2000017530CE75316012060B80127408F9748D
:102B3000AAF8752F017530CE75316812060B741323
:102B400078B2F6122B79222057147408F974AAF877
:102B5000752F017530CE75317012060B8012740816
:102B6000F974AAF8752F017530CE75317812060BFD
:102B7000741478B2F6122B792278ABE61201584021
:102B800004741ED32278ACE61201A8400C741FD343
:102B900022125E391200D7C32278AAE660F9B4FF88
:102BA00008D264756805022DF0B4021220380312B1
:102BB00027CE78B2E612756B400280DB80D3B40971
:102BC0000CC0E07404127031D0E0022DF0B438086B
:102BD00078ADE6122E0380BFB4390878ADE6122E28
:102BE0000D80B4B43A273068221227CE78AEE2784E
:102BF000AFF278B286F0E5F0543F4480C2AF75186A
:102C0000C0751909F51A120BD48086808AB43B244A
:102C10003068F81227CEE478AFF278B286F0E5F0AB
:102C2000543F4440C2AF7518C0751909F51A120B0C
:102C3000D4022B91B43C0C1227CE78B2E61276F96E
:102C4000022B91B43D391227CE203E18D23EC26DE0
:102C5000C2AF75187075190F751AE9120BD4757714
:102C600003022B91C23ED26DC2AF75186075190F69
:102C7000751AE9120BD47577031243FB022B91B43A
:102C80003E13E5715410600A1227CEE4122E120290
:102C90002B91022B97B43F14E5715410600B12274F
:102CA000CE74FF122E12022B91022B97B4400C12FD
:102CB00027CE78B2E61275EA022B91B4410C1227A6
:102CC000CE78B2E612764D022B91B4420C1227CE8A
:102CD00078B2E612762C022B91B4430C1227CE78F0
:102CE000B2E612760B022B91B4440E7400127031CE
:102CF00078B2E6128954022B91B4450E740012701A
:102D00005D78B2E6128965022B91B446097400120F
:102D1000707A40E880D5B4470E740212703178B2F0
:102D2000E6128976022B91B4480E740212705D7817
:102D3000B2E6128987022B91B44909740212707AA3
:102D400040E880D5B44A0E740312703178B2E612AE
:102D50008998022B91B44B0E740312705D78B2E621
:102D60001289A9022B91B44C09740312707A40E8BD
:102D700080D5B44D1A1289BA78B2E6543F4480C265
:102D8000AFF51A75190B7518C0120BD4022B91B43C
:102D90004E0C303E061227CE022C64022B91B44F0B
:102DA00009203EF71227CE022C4CB4540B74007845
:102DB000B24612889B022B91B45504744080F0B443
:102DC0005604748080E9B4570474C080E2B4580B90
:102DD000740078B246128885022B91B4590474406D
:102DE00080F0B45A04748080E9B45B0474C080E25B
:102DF0001227CEC2AF7518C0751907F51A120BD479
:102E0000022B9712766E78B2E678AAF222127678C2
:102E100080F4786CF208F212286E78B2E6543F44DF
:102E2000C0C2AFF51A75190B7518C0020BD4700526
:102E3000755F1E8002D21522C298C299322018F8FE
:102E400030991EC2992047057534008014C0F0C027
:102E5000E0C0D075D010E53412317BD0D0D0E0D0B6
:102E6000F020980132C2982047FAC0F0C0E0C0D0EC
:102E700075D010304605C246754000E54424FE403A
:102E800003754402E54020E72520E61FE54054078E
:102E9000232431C0E074003430C0E0E599220540BD
:102EA0002543F543D0D0D0E0D0F0320234F6543F81
:102EB00023232432C0E07400342FC0E0E5992215AA
:102EC0005E80DB80D9D55EFBB54312D213E8C0E04B
:102ED00078A274FAF2D0E0F875400080C702304161
:102EE000B462FA80B980B7B42AF380B2F55E24C622
:102EF000E55E40E924F5E55E50E3055E80A0781AC2
:102F0000F2155E8099781BF2155E8092781CF2159E
:102F10005E808B781DF2155E8084781EF2155E024D
:102F20002E9E781FF2155E022E9E7820F2155E020C
:102F30002E9E02306500022EE000022EE500022ED9
:102F4000E700022EEC00022EBF00022EBF00022E70
:102F5000BF00022EBF00022EFE00022F0500022F2E
:102F60000C00022F1300022F1A00022F2200022F42
:102F70002A00022EC500022EC500022EC500022E18
:102F8000C500022EC500022EC500022EC500022E6D
:102F9000C500022EC500022EC500022EC500022E5D
:102FA000C500022EC500022EC500022EC500022E4D
:102FB000C500022EC500022EC500022EC500022E3D
:102FC000C500022EC500022EC500022EC500022E2D
:102FD000C500022EC500022EC500022EC500022E1D
:102FE000C500022EC500022EC500022EC500022E0D
:102FF000C500022EC500022EC500022EC500022EFD
:10300000C500022EC500022EC500022EC500022EEC
:10301000C500022EC500022EC500022EC500022EDC
:10302000C500022EC500022EC500022EC5000230CA
:1030300065800E8039803D80418044804780548087
:1030400052B40909754300754000022E9EB421094F
:10305000754300754040022E9EB4420975430075C9
:103060004080022E9E754300754000022EA4B51EBE
:10307000D0022E9EB51FCA022E9EF541022E9EF54D
:1030800042022E9EB543BA75442012309575400019
:10309000022EA480D0854136126474D247E536B43E
:1030A0004603024C2CB4470412648A22B4500E85A5
:1030B000423512644FC2ACC247756B0722B453123B
:1030C000854235E542700A12644FC2ACC247756B47
:1030D0000222B4540E85423512644FC2ACC2477509
:1030E0006B0122B4550E85423512644FC2ACC24703
:1030F000756B0322B4560E85423512644FC2ACC2C2
:1031000047756B0422B4570E85423512644FC2AC2A
:10311000C247756B0522B4580E85423512644FC202
:10312000ACC247756B0622B44E3D854235E542B4CC
:10313000000B12644FC2ACC247756B0822B4010B7E
:1031400012644FC2ACC247756B0922B4020B126401
:103150004FC2ACC247756B0E22B4030B12644FC250
:10316000ACC247756B0F2224BF24E640048542356C
:1031700022C24722C5372537C53722E53424F0401F
:103180000EE53423249AC0E074003431C0E0227587
:103190009906C247753400D2B622802F803480361B
:1031A00080388039803E804680488051804F804DF5
:1031B000804B80468050800E023242753403F59970
:1031C000123174053422E5350231F075370074038D
:1031D00080ECE51E80E8E51F80E402329EE537754D
:1031E000340F80DA120C12122E2E883580D0E5357D
:1031F00080C9E535A23E92E080C1753403A835054B
:1032000035E676FF80B8E535C313603214700BA243
:103210002592E0B392E1440480D614700BA226926A
:10322000E0B392E1440880C8147008A22792E044F9
:103230000C80BD147008A20392E0440C80B274FCB0
:1032400080AEE535147025740830541230550444AE
:1032500006809D3056044403809644078092A25510
:1032600092E0A25692E1A22892E280841470157432
:1032700010A22592E0A22692E1A22792E2A2039256
:10328000E30231F014700D7418A21A92E0A21B929E
:10329000E10231F01470030231F0E40231F0E5365E
:1032A000B441067534040231BEB44212E535600300
:1032B000301503120C2A755F1E74420231BBB444F0
:1032C0000280F8B44B02800302335FE53554F8B452
:1032D000083AE5355407700A74191275EAE53602A2
:1032E0003396B4010A741912760BE536023396B49C
:1032F000020A741912762CE536023396B4030A7466
:103300001912764DE53602339602318FB42003024E
:10331000318FB42826E53520E008303E0B1243FB00
:103320008006203E03126698E535A2E0923E75675E
:10333000015003756702E5360231BBB4300CE53548
:1033400054F8127031E5360231BBB4380CE535540F
:10335000F812705DE5360231BB02318F02318FB455
:10336000430FB535037545037534077535CE023106
:10337000BEB44A28E535702120561E205408741921
:10338000126099126087C2AF75181075190F751AFF
:10339000F0120BD4E5360231BB02318FB44506750D
:1033A00034060231BEB4510675340C0231BEB44D40
:1033B0000EE5351273F6E5365002B2E70232BBB4C1
:1033C0004C0675340E0231BEB4460280C9B44702C1
:1033D00080C4B44F071289BA744F80BAB45917E544
:1033E000357013E8C0E078A4E2F535D0E0F8745900
:1033F00075340D0231BE02318FE56BB4000122C27B
:10340000AC128938128938D299E56BB407061234A8
:1034100093023477B4010612126E023477B40306B5
:103420001212F3023477B4020612118F023477B409
:1034300004061211D1023477B405061202DD0234FB
:1034400077B4060612133B023477B40806125F27DE
:10345000023477B40906125EAB023477B40E06125A
:103460005FB4023477B40F06125FFB023477B410F6
:103470000612359F023477C247D2B612644F756B7D
:103480000022E56BB4000122C247D2B612644F7528
:103490006B0022126250C2B67537007403124BAC37
:1034A000E51E124BACE51F124BAC7450124BAC74C2
:1034B0007D124BAC900000E535600F9003E814607E
:1034C000099007D0146003900BB87E7D7F0875F0DB
:1034D00000C0F0126250B40203D38001C3D0E033C5
:1034E000F5F0A3DFEC124BACDEE2E537124BAC306B
:1034F00099FD2202306520E5FA20E4F7540F2324D9
:103500000CC0E074003435C0E0E5992280E5801FEE
:1035100080238027802A803B803980378035803324
:103520008031802F802D802B80298043023041B54F
:103530001EFA022E9EB51FF4022E9EF541022E9E0B
:10354000F542600924F5E54240E2022E9E75404EA8
:10355000022E9EF5F0E54024BBC0E02410F8E5F013
:10356000F2D0E005E06542F8E5F0B800E380DEB5B2
:1035700043BA75442075400012644FC2ACC247750F
:103580006B10022EA4854236753500800EE542444C
:1035900080F53675350174017810F212361822E57F
:1035A00041B4284AE54224FD50E3C082C08378102C
:1035B000E2F58308E2F58208E2B4030A74191244C2
:1035C000071262278022B4020A741912443612616B
:1035D000A68015B4010A741912443F1261FE8008D6
:1035E000741912444812617DD083D0828097B42927
:1035F00025E54224FE5096C082C0837810E2F58310
:1036000008E2F5821262507812F27535038542366F
:10361000D083D08280858086C2B67537007423122D
:103620004BACE51E124BACE51F124BACE536124B12
:10363000ACE535124BACE535600E7810E2F5F0E5FF
:10364000F0124BAC08D535F4E537124BAC3099FD90
:1036500022E560C25B6002D25B855051789E76FFA6
:10366000C26EC240204A0C20481B304903023790EA
:10367000023CF01201027848E2F58308E2F582127A
:103680001BB702380B120102121E18121CA260197D
:10369000121D32603D1227CEC2AF75182075190F6A
:1036A000751AEC120BD40236D512449CB4020612E1
:1036B0003C43023CF0B4031AC082C0831200E412FF
:1036C000229FD083D08230490CE53C6008121B3E1B
:1036D000700302380B75483CD54519C2AF7518C048
:1036E000751900751A53120BD4754503757500745E
:1036F00006127031023CDBD2647568051227CEC217
:10370000AF7518C0751900751A07120BD4754F04E0
:103710001227A21227B875F06412011E023CF02095
:103720005724E573540860CC300C18C0E0C082C048
:10373000837411120188D083D082D0E0400280B718
:10374000023767023767E572548060A8300C18C0F2
:10375000E0C082C0837410120188D083D082D0E090
:1037600040028093023767127743401E205615307F
:103770002C03203E09900FE9123D18023CF0123C48
:103780006D023CF0123C73023CF0123C79023CF0BA
:10379000120102E53C608878C6E6B40A030243EDF4
:1037A000121D7B703912449CB40106123C43023C4A
:1037B000F0B403241200E4C082C083122334D08307
:1037C000D082304816C082C083120102121E18D067
:1037D00083D082121A26700302380B0236D578592C
:1037E000205802785AE2B40F0A124070C249D248F7
:1037F000023688B4100280F11227CEC2AF751820AD
:1038000075190F751AEB120BD480D030572D300C70
:1038100019C0E0C082C083740C120188D083D082AA
:10382000D0E0400302383B02382A756D02785BE233
:10383000785DF212417750030236D530582D300CA6
:1038400019C0E0C082C083740D120188D083D08279
:10385000D0E0400302386B02385A756D03785CE2A1
:10386000785DF212417750030236D5126643400369
:10387000122435E53B047011C2AF751820858319F9
:1038800085821A120BD40236D5754800754503742B
:103890000712705D740612705D2040057405127089
:1038A0005DC082C083123E4BD083D0825006123C52
:1038B00088023CF0C082C0831207EBD083D08250D4
:1038C00006123C88023CF0E58224CEE58334FF50AA
:1038D00043123DAB403E1287B85006123C79023C81
:1038E000F0023B7E123C79023AB4123C73023AB4C5
:1038F000123C6D023AB4123DB4500F123F3530E124
:1039000009302C24123C6D023CF01287B840F2D2F0
:103910006E023B7E12774340CB2056CE303E09E507
:1039200074542070D1202CC8305703784FE230589F
:1039300002E53B1201585009023982123C67023AF3
:10394000B4300CF7303BF41242DB4036A257303C27
:1039500001B3502E300C18C0E0C082C0837409122D
:103960000188D083D082D0E0400280CF02396FC07E
:1039700082C0831262A4D083D0825006123C7E02A1
:103980003AB4789D76FFD237300C19C0E0C082C0BF
:10399000837414120188D083D082D0E040030239AE
:1039A000A60239A4C2371242DB5003023A35A257AD
:1039B000303C01B3920A50161262FA5011303708A7
:1039C000126250B402028006123C55023AB41262EE
:1039D00050B40005200A2A8046B4013D200A223056
:1039E0001653757B10C2AF7518C0751900751A098A
:1039F000120BD4203706123C83023AB4123D6E807B
:103A000034E57454107009124451789E7602802572
:103A1000124451789D7602801CB402DA200AC0E577
:103A20007454107009124451789E76018007124434
:103A300051789D7601300C5C1242DB4057300C19F6
:103A4000C0E0C082C0837408120188D083D082D0C5
:103A5000E04003023A94023A59205B1CA257925A62
:103A600078A0A68378A1A682123D6AC257C25812D6
:103A700000F8756002023CF0756000E58378A0668E
:103A8000F5F0E58278A16645F07006123C8D023AA9
:103A9000B4124378123D18E57454106006300F03D9
:103AA00012445CE5715410600BC082C083123F5B0E
:103AB000D083D082E5745420600C306E0975F0C854
:103AC00012011E023CF0123DB45009123F3530E1A4
:103AD00003023CF01287B840F8C2A1D250D2A4C26F
:103AE0004F754F001227A21227B8121BB7C082C011
:103AF00083E57454807006122334023B5012232D48
:103B000030484D121A2670481200E475F064120114
:103B10001E12232D304839121A2670341200E47513
:103B2000F06412011E12232D304825121A2670202F
:103B30001200E475F06412011E12232D3048111298
:103B40001A26700C1200E475F06412011E12232D67
:103B5000D083D082204A0920481720491C023CF01B
:103B60001201027848E2B5830D08E2B58208023BF3
:103B70007E121A266008023CDB121B3E70F8789E0B
:103B800076FF300C19C0E0C082C083740612018831
:103B9000D083D082D0E04003023CDB023B9EE57143
:103BA0005401601FE58245836019305703784FE266
:103BB000305802E53B1201585003023BC3123C5BF4
:103BC000023CF0A23E926D127756500F123C617586
:103BD000F01E12011E1200C1023CF0B23E1227CEAE
:103BE000303E22C2AF75187085831985821A120B78
:103BF000D4757703C2A3C24ED2A1C250D2A4C24F81
:103C00001266988038C2AF75186085831985821A4C
:103C1000120BD4757703D2A3C24ED2A1C250C2A454
:103C2000C24F1243FBE57454206012E58224CEE5B6
:103C30008334FF5005123DAB50030239281200D7E0
:103C4000023CF0125E2F023C90125E2F023C90125A
:103C50005E2F023C90125E2F023C90125E2F023CBF
:103C600090125E2F023C90125E2F023C90125E2F4B
:103C7000023C90125E2F023C90125E2F8012125E68
:103C80002F800D125E2F8008125E2F8003125E2F90
:103C900075600078A076FF78A176FFD26B1227CEF0
:103CA000C2AF75182085831985821A120BD41200B1
:103CB000C1C26B22E5725408700320571DE5500401
:103CC000601814F5F07850E265F0600EC2AF751818
:103CD000C075190185501A120BD422125E2FD26BB7
:103CE0001200ABC26B75600078A076FF78A176FFFA
:103CF000C249C248E551F550789EE6B4020A741CE8
:103D00001244361261A6800BB40108741C12443FA1
:103D10001261FE789E76FF22303E0EC2A3C24EC2D2
:103D2000A2C251D2A4C24F800CD2A3C24EC2A2C220
:103D300051C2A4C24FA257920ED20D125E2F741C14
:103D4000126099126087E5715440600620A8031242
:103D500087DF1227CE123CB4C2AF751810858319C5
:103D600085821A120BD41200D722125E2F22125E05
:103D70002F75F03212011E227408F974AAF8752FFB
:103D80000175300375319012060B78AFE6085608BE
:103D9000560460141200E412229F304909E53C6089
:103DA00005121B3E6002C322D32222E582249CE539
:103DB0008334FF22E582249CE58334FF22E58225BB
:103DC00082F582E5833583F583E5822582F582E5F8
:103DD000833583F583E5822400F582E583345BF542
:103DE000837404F97400F8752F018583308582315E
:103DF0001205E62278AFE654C0F58378B0E630E4E9
:103E000002240A2323543C4583F58378AFE6C45447
:103E10000375F00AA4F5F0E6540F25F0030303F54B
:103E2000F053F0E085F08254034583F58378AEE6E5
:103E3000C4540375F00AA4F5F0E6540F25F045824A
:103E4000F58222C39582E5F09583221242DB50036E
:103E5000023ED3123DBD7800E2B4FF03023ED3120E
:103E60006992123DF478AAA68308A6827800E2F54A
:103E70008308E2F58208E2F5F008E2123E43502B97
:103E80007800E2F58308E2F58278AA86F008E61267
:103E90003E4350417802E2F58308E2F58278AA8633
:103EA000F008E6123E43402D023ED37800E2F5834F
:103EB00008E2F58278AA86F008E6123E43401678BA
:103EC00002E2F58308E2F58278AA86F008E6123E5F
:103ED000435002C322D322C3E58233F582E5833304
:103EE000F583E5822400F582E583349AF583740234
:103EF000F9744EF8752F018583308582311205E6FD
:103F000022C3E58233F582E58333F583E58224001D
:103F1000F582E583349AF5837402F9744EF8752FAF
:103F20000185833085823112058422784E7400F237
:103F300008E4F2801E300CF3C082C083123ED7D05A
:103F400083D082E5822418E58334FC4006784EE273
:103F50004402F2784FE2F5F018E222E5822400F5FF
:103F600082E58334BAF5837401F974AAF8752F01D8
:103F700085833085823112060B78AAE660422323BE
:103F8000C0E05403F5F0D0E054FC2400F582E5F0E5
:103F900034CAF5837404F974AAF8752F0185833047
:103FA00085823112060B78AAE60886F0786CF20852
:103FB000E5F0F275F002128908D5F0FA12286E22A7
:103FC00074FF786CF208F280EA7836E2540FC4F598
:103FD0008308E2540F428308E2540FC4F58208E2DA
:103FE000540F4282E5822460E58334F022783075F4
:103FF000F006E2540F08D5F0F9E2540F75F00AA468
:10400000F58275830008E2540F2582F582E58275FA
:10401000F00AA4F58285F08308E22582F582500239
:104020000583E58275F00AA4F582C0F0E58375F09A
:104030000AA4D0F025F0F58308E22582F58250022B
:104040000583E5822460E58334F022D3227830E2D0
:10405000600BF5F008E2240A4005D5F0F7C322D33F
:1040600022783079BA75F00AE2F70809D5F0F9221A
:10407000C082C08378BA9002DC75F00AE0F608A32B
:10408000D5F0F99002E6E0F56AD083D08222C082B2
:10409000C08378BA9002DC75F00AE6F008A3D5F088
:1040A000F9E56A9002E6F0D083D0822212406112D4
:1040B0001A2622D083D0822212406112408E12230F
:1040C0000DC082C083753C0175F0057830E2540F55
:1040D00070E108D5F0F7E208540FF9E208540FC474
:1040E000F5F0E208540F45F0FAE208540FC4F5F079
:1040F000E208540F45F0FB1203D6EC70B678C6C246
:1041000061EDC4124128ED124128EEC4124128EE9F
:10411000124128EFC4124128D261EF124128E8244D
:104120003AF53CD083D08222540F7003306104D220
:1041300061F6082279C677000975F00577FF09D581
:10414000F0FA2212406112408E12413475F0087864
:1041500032753C06E2540F700608D5F0F7800979F5
:10416000C6E2F70809D5F0F922124143121B3E229C
:104170001240B8121B3E22785DE2700302423924DD
:10418000FD4038C082C0831200E4124295D083D033
:1041900082204A1620490B304836121A2670310206
:1041A0004239121B3E70290242397848E2B5832019
:1041B00008E2B5821B65827017807EE224E2407DB2
:1041C000C082C0831200E4126BB5D083D08250034A
:1041D00002423B785DE2B40F0C124169605B124011
:1041E000AC605680EBB41007124170604C80E1B4B3
:1041F000110AC082C083123FC902422075F00384B5
:10420000E5F0B4000712416970C6802DB4010712B1
:1042100040AC70BC8023B4021EC082C083123FED4C
:10422000E5828583F0D083D08240A5658270A1E5C8
:10423000F06583709B80028097C322D322C082C026
:10424000831200E4126C02D083D0825002D3227811
:104250005DE275F00384E5F0B4000A1242E9121B36
:104260003E70EA802CB4010A124311121A2670DD46
:10427000801FB4021EC082C083124314E58285836E
:10428000F0D083D08240C6658270C2E5F06583704D
:10429000BCC32280B8754732D253304C09C24CC0DF
:1042A0006D12027AD06DE547D36018C24AC249C286
:1042B0004812216E50E4122995204A062049033005
:1042C00048D8C3C0D0A86D7405B802027404D0D019
:1042D0004005122948800312297022E582B4E807BC
:1042E000E583B40F02D322C32212404D5002D322E1
:1042F0007830E260F9F5F008753C06E2540F70067C
:1043000008D5F0F7800979C6E2F70809D5F0F9C3B6
:1043100022026D2412404D5004D322C3227830E291
:104320000860F6B40108E2F58275830080EDB402FE
:1043300012E275F00AA4F58208E22582F5827583FF
:104340000080D8B40320E275F00AA4F58208E225C3
:104350008275F00AA4F58285F08308E22582F58251
:1043600050B9058380B5B404057831023FF9C39490
:1043700004F5F07831023FF2B257B258754F071288
:1043800027A21227B8B258B257C2AF7518C0751914
:1043900000751A0C120BD4305A0EC2AF7518B075D6
:1043A0001900751A00120BD4123CB4C082C0837875
:1043B000A0868378A18682C2AF751810858319857F
:1043C000821A120BD4D083D08222E53CB4031C782D
:1043D000C6E6B40A1608E624F6401008E624F640BD
:1043E0000A18E675F00AA40826C322D3221243CA8B
:1043F00050030237A078A8F2024507126698128986
:10440000BA1244B3C2402230162B543F44C0C0827B
:10441000C083C0E0C2AF7518E085831985821A1287
:104420000BD4D0E0C2AFF51A75190E7518C0120B77
:10443000D4D083D082223016FC543F448080CF30C9
:1044400016F3543F444080C63016EA543F4400807F
:10445000BD78A5E582F278A6E583F222789DE6B4E0
:104460000118C082C08378A5E2F58278A6E2F583C0
:10447000741C12443F1261FE8019B4021AC082C03B
:104480008378A5E2F58278A6E2F583741C1244369F
:104490001261A6D083D082789D76FF2220570AE44D
:1044A000A26F92E0A27092E122E4A27192E0A27265
:1044B00092E122740712705D740612705D74051229
:1044C000705D22455E458045BC45324532453245EA
:1044D0003245E845F6460446124620465C4690467C
:1044E0009846AA46B846F6474A476F478647A947BF
:1044F000C747E547F1480F482D48394857487548A0
:1045000081489C4B204B5678A8E224DE4024124A76
:104510003E401378A8E225E0049044C393C0E0E253
:1045200025E093C0E022024AF8124AF71200D702AF
:104530003CF0740A024AF8D2A1C250C2A4D24F126F
:104540004AF61200E4122334204902D322E53CB497
:1045500002F978C6E624F640F208E624F622124A6A
:10456000F5124537401578C6E62430F51E08E624D6
:1045700030F51F121A001258EE80AE7420024AF86D
:10458000124AF51249DD402F12699278C6E6C40836
:1045900046F5F078CAE65403030345F078AFF678A1
:1045A000C8E6C40846F5F078CBE6C42345F078B0F9
:1045B000F6126944024529741E024AF8124AF5129D
:1045C000498E401F12699278C6E6C4084678AEF656
:1045D00078C8E6C4084678ADF6E478ACF6126944CB
:1045E000024529741F024AF8124AF5124AD7741B71
:1045F0001275EA024529124AF5124AD7741B12763F
:104600000B024529124AF5124AD7741B12764D0245
:104610004529124AF5124AD7741B12762C024529F5
:10462000124AF51287B8402F124AD712669812899B
:10463000BA1244B3C240C23ED26D7848E2F5830854
:10464000E2F582C2AF75186085831985821A120B54
:10465000D47577030245297416024AF8124AF512F6
:1046600087B840F312775640EEC26D124AD71266F1
:1046700098D23E7848E2F58308E2F582C2AF751819
:104680007085831985821A120BD475770302452928
:10469000124AF5203E8A80C4124AF5124AD775F0B4
:1046A000C8128908D5F0FA026613124AF5124AD7E1
:1046B000741B1276F9024529124AF520170D12498A
:1046C00056402E124B0B402978A9F278A9E2F550FA
:1046D000F551124AD7C2AF7518C085501A75190323
:1046E000301703751902120BD40245297419024AB6
:1046F000F8741A024AF8124AF520170D124956406A
:10470000F0124B0B40EB78A9F278A9E2F550124A6F
:10471000D7C2AF7518C085501A75190630170375C2
:104720001905120BD4125B99125BD0123DAAD2A2CA
:10473000C251C2A1D2501200E4122334741820488E
:1047400006204903304AAC023664124AF530682F1D
:1047500078AEE278AFF2124AD7741B543F4480C25D
:10476000AF7518C0751909F51A120BD40245291234
:104770004AF530680A124956500A741C024AF87405
:104780001D024AF870CD124AF53068F3E478AFF2B2
:10479000124AD7741B543F4440C2AF7518C07519F4
:1047A00009F51A120BD4024529124AF57400127049
:1047B00031741B543F4400C2AF7518C075190AF517
:1047C0001A120BD4024529124AF5740012705D7456
:1047D0001B543F4480C2AF7518C075190AF51A12F0
:1047E0000BD4024529124AF5740012707A40DB801E
:1047F000BB124AF57402127031741B543F4400C25C
:10480000AF7518C075190CF51A120BD40245291290
:104810004AF5740212705D741B543F4440C2AF7578
:1048200018C075190CF51A120BD4024529124AF555
:10483000740212707A40DB80BB124AF57403127066
:1048400031741B543F4480C2AF7518C075190CF504
:104850001A120BD4024529124AF5740312705D74C2
:104860001B543F44C0C2AF7518C075190CF51A121D
:104870000BD4024529124AF5740312707A40DB808A
:10488000BB7404127031741B543F4440C2AF75189E
:10489000C075190BF51A120BD40245291289BA7486
:1048A0001B543F4480C2AF7518C075190BF51A121E
:1048B0000BD4024529C2A1D250C2A4D24F123DAAA4
:1048C0001200E4122334204A0920481F20495102D3
:1048D00048E97848E2F58308E2F582120102300CDB
:1048E00006123F3520E202C322D322121CA270F925
:1048F00012449CB4020280F1B4031AC082C0831235
:1049000000E412229FD083D0823049DDE53C60D99B
:10491000121B3E70D47848E583F208E582F280BB32
:10492000121D7B70C412449CB4010280BCB40324E9
:10493000C082C0831200E4122334D083D082304876
:10494000A8C082C083120102121E18D083D0821226
:104950001A26709580BFD2A1C250C2A4D24F124A6B
:10496000F61200E4122334204902D322E53C60FA17
:1049700024FC40F6A93C78C67A00EA75F00AA42621
:1049800040E8C5F070E4AAF008D9EFEAC322D2A14A
:10499000C250C2A4D24F124AF61200E412233420AD
:1049A0004902D322E53CB404F9F5F078C6E624F6D2
:1049B00040F008D5F0F778C6E675F00AA40826247A
:1049C000E8402E78C8E675F00AA4082624C44021E1
:1049D00022E0E2E0E1E0E1E0E0E1E0E1E0D2A1C2FA
:1049E00050C2A4D24F124AF61200E41223342049D6
:1049F00002D322E53CB406F9F5F078C6E624F64089
:104A0000F008D5F0F778C8E675F00AA4082660E14A
:104A1000C0E024F3D0E040D99049D093F978C6E6BD
:104A200075F00AA4082660C9C0E029D0E040C27829
:104A3000CAE624F640BB78CBE624F940B422300C19
:104A40007C7848740FF20874E9F220177C78A8E2A9
:104A50002400F5827583D07401F974AAF8752F01CA
:104A600085833085823112060B78AAE612015850F0
:104A70006278A8E22400F5827583D17401F974AAE2
:104A8000F8752F0185833085823112060B78AAE6EE
:104A90001201A8503678A8E22400F5827583CF74FD
:104AA00001F974AAF8752F018583308582311206C9
:104AB0000B78AAE620570C20E01530E10C1248B51F
:104AC000740D2220E20920E3F4C322740E800674E0
:104AD0000C8002740BD32220171A1227CE7848E2DA
:104AE000F58308E2F582C2AF7518E08583198582E7
:104AF0001A120BD422222222C0E0125E2F124AF593
:104B0000D0E0125A121200AB023CF0C050C082C07A
:104B100083F550125A95D083D082E550D050B322FD
:104B2000124AF5D2A1C250C2A4D24F124AF61200C4
:104B3000E4122334204902D322E53CB401F978C6BB
:104B4000E654FC70F2E60303441CC0E0124AD7D0DE
:104B5000E0128885C322124AF5D2A1C250C2A4D263
:104B60004F124AF61200E4122334204902D322E500
:104B70003CB401F978C6E654FC70F2E60303441C29
:104B8000C0E0124AD7D0E012889BC322C537253730
:104B9000C53722E54824E94008D2A3C24ED2A2C2BA
:104BA000513098EFC298E599124B8C223099FDC292
:104BB00099F599124B8C22C2A3C24EC2A2C251C215
:104BC000B67537007405124BACE51E124BACE51FF1
:104BD000124BAC22128938128938128938124BB71D
:104BE000E536124BACE537124BAC3099FD22120B77
:104BF00042024BF7120ADEC0E0124BB7E536124B09
:104C0000ACD0E0124BACE537124BAC3099FD221220
:104C10008938124BB7E536124BAC797CE7124BACB6
:104C200009DDF9E537124BAC3099FD22D2187548F1
:104C300019751A001289BAE538600B54F87007C26A
:104C400029A229B392A5E539600B54F87007C22A4E
:104C5000A22AB392A6E53A600B54F87007C204A2E8
:104C600004B39280126094C28EC28CC2ADC2ABC239
:104C7000ACC2AF7581D3904C81C082C08375D00027
:104C800032D2AFD28C12644FC2ACD299124BD4B292
:104C9000B5754819D298024CBEB40922F537124BAB
:104CA00093B51E27124B93B51F21124B93B4461B8D
:104CB000124B93AF37124B936F7010124BD4D2B686
:104CC000D2A3C24ED2A2C251124B93B40ACBF53733
:104CD000124B93B51EF5124B93B51FEF124B93F584
:104CE00036B46D03024D6EB46E03024D87B46F038C
:104CF000024DBEB47003024E0BB47103024E1FB4DA
:104D00007303024E30B47403024E32B47503024E84
:104D100046B47603024DBBB47703024E5EB478030B
:104D2000024E72B47903024E93B47A03024EAFB4CA
:104D30006C03024EC3B46B03024EE5B46A03024F28
:104D400020B46903024F3CB46803024F98B4670370
:104D5000024FB0B46603024FCBB4650302508FB468
:104D6000630302579AB46103025805024CBEAF3781
:104D7000124B936F70F5124BD4D2B675F01E128998
:104D800008D5F0FA026613124B93FD1424E0402B71
:104D9000124B932400FC7B00124B93FEAF37124B57
:104DA000936F70178EF0EDF9747CF88B2F8C308533
:104DB000F03112060B124C0F754819024CBE124B03
:104DC00093FD1424E040F4124B932400FC24714022
:104DD000EA7B02124B93FEEDFA787C124B93F608B5
:104DE000DAF9AF37124B936F70D1C2A3C24EC2A291
:104DF000C2518EF0EDF9747CF88B2F8C3085F03138
:104E00001205B5124BDD75481980B0AF37124B93C0
:104E10006F70A8120902124BD4754819024CBEAF2C
:104E200037124B936F7009124BF4754819024CBE40
:104E30008089124B93FD1424E04034124B932400DC
:104E4000FC7B01024D98124B93FD1424E04020128C
:104E50004B932400FC242540167B03024DD3AF372F
:104E6000124B936F7009124BEE754819024CBE023B
:104E70004DBB791A7D07124B93F309DDFCAF371256
:104E80004B936F70EA125A1440E5126944124BDDDD
:104E9000024CBEAF37124B936F70D41269921289D5
:104EA00038124BB7E536124BAC1202F9024CBEAFCA
:104EB00037124B936F7066120F21124BD47548193D
:104EC000024CBE124B93FE124B93FD124B93FCAF60
:104ED00037124B936F70461208684041124BD475DD
:104EE0004819024CBE124B93FE124B93FDAF371282
:104EF0004B936F7028120839128938128938124B77
:104F0000B7E536124BACEE124BACED124BACEC12DB
:104F10004BACE537124BAC3099FD024CBE024DBB99
:104F2000AF37124B936F70F5128938128938124BD4
:104F3000B7E536124BAC121354024CBEAF37124BCE
:104F4000936F70D9120AD660027401C0E0120B3A56
:104F500060027402D0F045F0700712094D12165E1F
:104F6000E4C0E0124BB7E536124BACD0E0C0E01223
:104F70004BACE537124BAC75F003128908D5F0FA4B
:104F8000124BB7E536124BACD0E0124BACE5371202
:104F90004BAC3099FD024CBE124B93FD1424E04003
:104FA00027124B932400FC2471401D7B00024DD33B
:104FB000124B93FD1424E0400F124B932400FC2469
:104FC0002540057B01024DD3024DBBAF37124B93F9
:104FD0006F70F5128938128938124BB7E536124BCB
:104FE000AC7402124BAC744E124BAC7484124BACCA
:104FF0007448124BAC7433124BAC7400124BAC744B
:105000008D124BAC7420124BAC74DA124BAC7400A2
:10501000124BAC740F124BAC74A0124BAC748012D8
:105020004BAC7400124BAC7400124BAC7420124B9E
:10503000AC7400124BAC7400124BAC7400124BAC4D
:105040007400124BAC7400124BAC7400124BAC7475
:1050500000124BAC7400124BAC7400124BAC7400D9
:10506000124BAC7400124BAC7400124BAC740012B7
:105070004BAC7400124BAC7400124BAC7400124B6E
:10508000ACE537124BAC3099FD024CBE024DBB1261
:105090004B93F583124B93F5822460E58334F04003
:1050A000EB12531B124B93FD1424E040DF78007584
:1050B000F02074FFF208D5F0FB7800124B93F20851
:1050C000DDF9AF37124B936F70C2124BD475F005F8
:1050D000128908D5F0FA124BDD751A01300CAD12A9
:1050E0005351125337125329121BB778BA79007AE9
:1050F0000A75F00FE3540FF652F00809DAF643F0A0
:10510000F0E5F00478C379AE7428121A37600B12F8
:1051100051B05006751A0402508C1253371253299D
:10512000121BB778C6790A7A0675F00FE3540FF6AA
:1051300052F00809DAF643F0F0E5F00478CB79B1E3
:105140007418121A37600B12524E5006751A060266
:10515000508C12533712539A751A65024CBEC0E038
:105160007830E583F208E582F2D0E022C0E07832C0
:10517000E583F208E582F2D0E022C0E07830E2F583
:105180008308E2F582D0E022C0E07832E2F58308BD
:10519000E2F582D0E022E5822400F582E583341B2B
:1051A000F58322E5822400F582E583343BF58322F2
:1051B000125329AB83AC82901B00C0837900752FFA
:1051C0000385833075310090005112056A12067A0A
:1051D00012056A1206C49000517A80E0A3F5F0E04F
:1051E000A36C7005E5F06B6017DAF0D0830583746B
:1051F0000024C0E58334C550C174051252FDD3228A
:10520000D083EA2AF5F0E4C395F0F58212515E7876
:10521000BA79007A0A75F00FE3540FF652F00809D4
:10522000DAF643F0F0E5F004600C121CA5700A7485
:10523000061252FDD322121CA5E5822582F582E5D5
:10524000833583F58312519612516C0255A2125385
:1052500029AB83AC82903B00C0837900752F038516
:10526000833075310090005112056A12067A1205DA
:105270006A1206C49000517A80E0A3F5F0E0A36CB6
:105280007005E5F06B6017DAF0D0830583740024B5
:10529000C0E58334A550C174051252FDD322D083DA
:1052A000EA2AF5F0E4C395F0F58212515E78C679EA
:1052B0000A7A0675F00FE3540FF652F00809DAF691
:1052C00043F0F0E5F004601D121D8B701BAB83AC46
:1052D00082125329EBB58306ECB58202C322740413
:1052E0001252FDD322121D8BE5822582F582E583C1
:1052F0003583F5831251A312516C0255A2F51A227F
:10530000C082C083E583125A13D083D082C082C08A
:1053100083E582125A13D083D08222C0E07834E52C
:1053200083F208E582F2D0E022C0E07834E2F5832F
:1053300008E2F582D0E0227400124BAC7400124BEC
:10534000AC7400124BAC7400124BAC7400124BAC3A
:105350002275831B75821B75F040C0F0C082C0832C
:10536000752F0185833075310012056A12067AD0D7
:1053700083D082C082C083752F038582307531004F
:1053800012056A120718D083D08205830582D0F0F7
:10539000D5F0C77532FF7533FF227401F97418F820
:1053A000752F0075300075310012060B7401F97409
:1053B00019F8752F017530D97531FF12060BAC182D
:1053C000125329E5822420F582E583347DF583C0DC
:1053D00082C0837401F9743BF8752F008583308592
:1053E000823112060BD083D0827401F97410F875E3
:1053F0002F008583308582311205847810E2F5F024
:10540000E518253BC395F0F518125329123ED778BD
:105410004E79AAE2F72519F5190809E2F72519F5D9
:10542000197816794EE2F3FA0809E2F32AFAC3E58D
:10543000199AF519125329123F01125329E5827561
:10544000F008A42420F582500205F0A8F0E5837549
:10545000F008A4282400F5837408F974AAF8752FBD
:105460000085833085823112060B78AAE5187A0808
:105470002608DAFCF51878BA79007A0A75F00FE395
:10548000540FF652F00809DAF643F0F0E5F0041292
:1054900059B078C6790A7A0675F00FE3540FF652C0
:1054A000F00809DAF643F0F0E5F0041259B8740890
:1054B000F974AAF8752F008583308582311205B5FD
:1054C00078AAE5187A08C39608DAFBF5181253296A
:1054D000C3E58233F582E58333F583C3E58233F593
:1054E00082E58333F583E5822400F582E583245B3E
:1054F000F583C082C0837404F974AAF8752F0185FE
:10550000833085823112060BD083D0827404F97403
:1055100012F8752F0185833085823112058478AAAF
:105520007912E5197A0426F5F0E3C5F0C395F00881
:1055300009DAF3F5197401F97418F8752F0075304C
:10554000007531001205B57401F97419F8752F0151
:105550007530D97531FF1205B575831B75821B75C2
:10556000F040C0F0C082C083752F03858330753151
:105570000012056A12067AD083D082C082C0837579
:105580002F0185823075310012056A120718D08309
:10559000D08205830582D0F0D5F0C77532FF753310
:1055A000FF22125188E5828583F012517AC39582D9
:1055B000C0E0E5F09583D0F045F07002C3225003BF
:1055C0000256BD125188C0E0C3E58224FEF582E593
:1055D0008334FFF583D0E012516CE5828583F012AD
:1055E000517AB58207E5F0B58302C32212517AAF32
:1055F00083125188EFB58310AE8290003478AAE010
:10560000F6A308E0F60256207EFE8F83058374021F
:10561000F974AAF8752F0385833075310012060BD3
:105620007900752F038F3075310090005112056A93
:1056300012067A12056A1206C48F8375820012510F
:105640007A7D00E5836F7002AD82ED2451F582759D
:10565000830050020583C3EE9D20E05A03FCC08204
:10566000C083A3A3E0FAA3E0FBD083D082EAF0A337
:10567000EBF0A3DCE9EE2451F582758300500205BE
:105680008378AAE6F0A308E6F07900752F038F303F
:1056900075310090005112056A12070412056A1252
:1056A0000718852F32853033125188EFB5830302F6
:1056B00057910F0255F174081252FDD32212517AFC
:1056C000AF83125188EFB58310AE8290003478AA70
:1056D000E0F6A308E0F60256F17E008F831583748E
:1056E00002F974AAF8752F038583307531FE12060E
:1056F0000B7900752F038F30753100900051120522
:105700006A12067A12056A1206C412517A7DFEE503
:10571000836F7002AD82ED2451F5827583005002D3
:105720000583C3ED9E20E06B03FCC0E0C3E582244B
:10573000FEF582E58334FFF583D0E0C082C083E0CC
:10574000FAA3E0FBA3EAF0A3EBF0D083D082DCDA8B
:10575000EE2451F5827583005002058378AAE6F0A5
:10576000A308E6F07900752F038F307531009000A3
:105770005112056A12070412056A120718852F32A2
:10578000853033125188EFB583030257911F0256BB
:10579000C2C32274091252FDD322124B93F5831215
:1057A0004B93F582124B937010124B93700BAF37E3
:1057B000124B936F70030257BC024DBBC01EC01F3B
:1057C00085831E85821F121A007401F974AAF87568
:1057D0002F0075300075310012060B78AAE6C395CC
:1057E0001EC3951FD01FD01E251E251FF67401F95C
:1057F00074AAF8752F007530007531001205B512C6
:105800004BD4024CBE124B93F583AF37124B936FC0
:1058100070A7128938128938128938124BB7E536C9
:10582000124BAC7400124BACE51A124BAC74001264
:105830004BAC7400124BAC7400124BAC7400124BA6
:10584000ACE537124BAC3099FD024CBE905854C0B9
:1058500082C083327581D375D000026613C082C0C6
:1058600083E5822420F582E583347DF5837401F994
:10587000743BF8752F008583308582311205B5D0D1
:1058800083D082C082C083E58275F008A42420F50D
:1058900082500205F0A8F0E58375F008A4282400E2
:1058A000F5837404F974AAF8752F00858330858216
:1058B000311205B5A3A3A3A37404F974AEF8752F30
:1058C000008583308582311205B5D083D082E58290
:1058D0004583600EE5822418E58334FC74FFF5F0FF
:1058E000500BC082C083123F01D083D08222120AA3
:1058F000DEC0E07401F974AAF8752F0075300075E8
:10590000310012060B78AAE6D0F0C395F0F67401C8
:10591000F974AAF8752F007530007531001205B5BD
:1059200022753B00784FE4F278AA75F00876FF08FC
:10593000D5F0FA22751E30751F30C257C25875F067
:1059400005C0F0D2A3C24EC2A2D251D2A1C250D23F
:10595000A4C24F125921122334D0F0204809204903
:1059600006D5F0DD0259AB1259D0403F1200D7786E
:10597000AFE6B4FF05C32275F005C0F0122334D0A2
:10598000F0204906D5F0F30259ABE53CB4021C788F
:10599000C6E624F6401508E624F6400F78C6E6244D
:1059A00030F51E08E62430F51FC3221200ABD322C7
:1059B00078BA79AA7A05800678C679AF7A03E608BC
:1059C000540FC4F5F0E608540F45F0F709DAEF225A
:1059D00020483130493AE53C600624FD24FC403043
:1059E0001259B81200E475F005C0F0122329D0F066
:1059F000204811203F06D5F0F0025A10121405B4C9
:105A00000B0E80031259B0753B00784FE4F2C322AD
:105A1000D3222222781FE254C07078E275F00A8403
:105A2000C445F078ACF6781EE254C07066E275F0BA
:105A30000A84C445F078ADF6781DE254E07054E273
:105A400075F00A84C445F078AEF6781CE2604454E0
:105A5000E07040E275F00A84C445F0C0E0781AE2D4
:105A6000030354C0D0F045F078AFF6781BE2602312
:105A700054F0701FE275F00A84C445F0C0E078204D
:105A8000E254F8700EE2C42354E0D0F045F078B050
:105A9000F6C322D32290000075F019C0F07402F909
:105AA00074AAF8752F0185833085823112060B7830
:105AB000ABB6FF02801318E550300C0AB4FF07881C
:105AC000F07850E2A8F0666011E5822410F582506B
:105AD000020583D0F0D5F0C3C322D0F0A3D3223087
:105AE0000C4DE58224FFF582E58334FFF58375F0E4
:105AF00019E5822480E58334FE5005900000800A79
:105B0000E5822410F58250020583C0F07402F97416
:105B1000AAF8752F0185833085823112060B78AB88
:105B2000B6FF02800518E6B55007D0F0D5F0C2C325
:105B300022D0F0A3D322120114300C0C125A95403B
:105B40000390FFF1125ADF22C050125B66D0502240
:105B5000300C13125A95400390FFF1125ADF500592
:105B6000F550125B9822E55070057550108023B4F3
:105B70001005755011801BB411057550208013B4A9
:105B800020057550FF800BB4FF057550008003752C
:105B900050FF125C49E550222230130CC213125AF6
:105BA000144005126944800312699278AFE6C45428
:105BB00003E6540F78B0E6C45401E6540F78AEE61D
:105BC000C4540FE6540F78ADE6C4540FE6540F22C8
:105BD000300C0A125A955005125B988003125C49EA
:105BE00022C2AC12644FC2AC128938128938D299E1
:105BF000C2B674FF124BAC7537007442124BAC74D2
:105C000062124BAC7415124BAC742A124BAC741B61
:105C1000124BAC7400124BAC7400124BAC740012FB
:105C20004BAC7400124BAC12030675F010C0F0744C
:105C300000124BACD0F0D5F0F4E537124BAC3099F4
:105C4000FDC247D2B612644F22222016012274757B
:105C5000787212012F501C205C1BD25C12611374ED
:105C60001A543F4400C2AF7518C075190BF51A12CB
:105C70000BD422C25C126992203104203235227882
:105C8000AEE6543FF5F07968E365F0702309E378F8
:105C9000AD66701C203318D233126113741A543F4E
:105CA0004400C2AF7518C075190BF51A120BD42237
:105CB00030323178AEE6543FF5F0796AE365F07042
:105CC0002309E378AD66701C203318D233126113B8
:105CD000741A543F4400C2AF7518C075190BF51AF9
:105CE000120BD422C23322C2AC120C12600CF51873
:105CF0008819120F94120C2A80EFD2AC227E007FFA
:105D00008C90000075F000E49325F0F5F0A3C3E556
:105D1000829EE5839F40F0E5F070022200E5F0C02E
:105D2000E0E583125A13E582125A13D0E0125A1397
:105D3000C2ADC2ACD218D2A3C24ED2A2C251C2A12D
:105D4000C250D2A4C24FC2A080EC300C4174007883
:105D50008212013E40387F087E007478787212010A
:105D60002FCE13CE05E0DFF420190F7400789212C5
:105D7000013E5006EE789C666014EE789CF6F55075
:105D8000C2AF7518C075190485501A120BD422C2FF
:105D9000AFF51A75190F751810020BD422300CFCD0
:105DA0002054F97401788212013E40F074777872C1
:105DB00012012FE492E0C0E07476787212012FD0C5
:105DC000E033FE20190F7401789212013E500678DC
:105DD0009FE66E60C7EE789FF620E10630E028026D
:105DE0005E1A30E014A256725550B1C256C2551216
:105DF000607374F8125D8F80A3D256C2551260731F
:105E000074F7125D8F809520550ED255C2561260E0
:105E100073D25374F6125D8F8082A228825540F8A7
:105E2000D255C25612608774F5125D8F025D9CC018
:105E300082C083D083D0822222303E09C2A3C24EC8
:105E4000D2A4C24F22D2A3C24EC2A4C24F22200C5F
:105E500001227473787212012FE492E0C0E074742E
:105E6000787212012FD0E092E1F5F0657853F003DB
:105E700085F0786009E5F00303441A12888574718F
:105E8000787212012FE492E0C0E07472787212010D
:105E90002FD0E092E1F5F0657953F00385F0796059
:105EA00009E5F00303441A12889B22C2B675370035
:105EB0007403124BACE51E124BACE51F124BAC74D5
:105EC0004E124BAC7408124BAC7401124BAC7406FE
:105ED000124BAC7843E2F5F0E5F0124BAC08E2F57A
:105EE000F0E5F0124BAC7845E2F5F0E5F0124BAC82
:105EF00008E2F5F0E5F0124BAC242AF8E27847E22C
:105F0000547FF5F0782CE2C36001D3E5F092E7F519
:105F1000F0E5F0124BAC75F000E5F0124BACE53754
:105F2000124BAC3099FD22C2B6126EF3126E82751E
:105F300037007403124BACE51E124BACE51F124B3D
:105F4000AC744E124BAC740C124BAC7400124BACD4
:105F5000740A124BACC082C083A3A3A3E49375F070
:105F600064A4C0E0E5F0124BACD0E0124BACA3A3AC
:105F7000A3A3E49375F064A4C0E0E5F0124BACD0A9
:105F8000E0124BACD083D082E493124BACA3E493E9
:105F9000124BACA3A3A3E493124BACA3E493124B18
:105FA000ACE58D124BACE58B124BACE537124BAC2C
:105FB0003099FD22C2B612149FC0E07537007403F9
:105FC000124BACE51E124BACE51F124BAC744E12DB
:105FD0004BAC7404124BAC7402124BAC7402124BF7
:105FE000AC78A4E2F5F0E5F0124BACD0F0E5F0129D
:105FF0004BACE537124BAC3099FD22C2B612141FE0
:10600000C0E07537007403124BACE51E124BACE5D3
:106010001F124BAC744E124BAC7404124BAC740296
:10602000124BAC7402124BAC78A4E2F5F0E5F0121E
:106030004BACD0F0E5F0124BACE537124BAC3099DD
:10604000FD22C0F088F0C0F0C2AF756E00784BE260
:10605000F54AF5F008E2F54BD2AF45F0D0F0A8F0E4
:10606000D0F07009B22820280412607D22D2287551
:106070006E0322C2AF754AFF754BFFD2AF756E003B
:10608000C20DC228D2A722126042D253D24D22C2E0
:1060900062027522D26202752230551420281154F2
:1060A0003F4400C2AFF51A7519087518C0020BD429
:1060B00022D2B2C2B4D293C322D2B2C2B4D2931209
:1060C000892020B2ECC29312892030B2E4D293121C
:1060D000892012892020B2D9C293128920128920E6
:1060E00030B2CED2B2C2B4D293D322120656C284F8
:1060F0007454120661E4120630120643F5F0644847
:10610000255A33F55AE5F0255BB2E003F55BD9E992
:10611000D284227583DD75F010752F038583307569
:106120003100C083C0F012056A120A70D0F0D0832B
:106130000583D5F0E47532FF7533FF756F00757018
:106140000022E5822400C0E0E58334DDF8D0E0C31E
:1061500022C082C0837401F974AAF8752F03858365
:106160003085823112060B78AAB6020CE57024FF46
:10617000F570E56F34FFF56FD083D0822212614253
:10618000C082C083F582888312615178AA76007438
:1061900001F974AAF8752F038583308582311205C1
:1061A000B5D083D08222126142C082C083F582883A
:1061B00083C082C0837401F974AAF8752F038583A4
:1061C0003085823112060B78AAB60209D083D082BC
:1061D000D083D08222E5702401F5705002056FD083
:1061E00083D08278AA76027401F974AAF8752F0315
:1061F0008583308582311205B5D083D08222126129
:1062000042C082C083F582888312615178AA7601E8
:106210007401F974AAF8752F0385833085823112D1
:1062200005B5D083D08222126142C082C083F5823C
:10623000888312615178AA76037401F974AAF875FB
:106240002F038583308582311205B5D083D0822219
:10625000126142C082C083F58288837401F974AAF6
:10626000F8752F0385833085823112060B78AAE6F4
:10627000B40102800CB402028007B40302800274ED
:1062800000D083D08222120656C284745412066152
:10629000E4120630120643B40205755A018002D991
:1062A000F3D28422755A007583DD75F00F752F03C4
:1062B000858330753100C083C0F012056A12067AFA
:1062C00012056A7900126286D0F0D0830583E55A00
:1062D0007026D5F0D8752F038583307531001205EF
:1062E0006A12067A12056A79A01262867532FF7503
:1062F00033FFE55A7002D322C322E570456F601662
:10630000785FE2F5F008E245F0600BD37860E29543
:106310007018E2956F22C322C28C758A45758C5D18
:10632000D28CB20020000132C0D0C0E0C0F075D0E5
:1063300008D24C121404126430051DE51D20E00C37
:1063400020E109301816E51D541F604A201804E5A5
:10635000496002B2B5D0F0D0E0D0D032205105A2D1
:1063600028B392A2E51D30E203127272E51D541F9C
:106370007027D24DC26678A3E2D5E006D265D26618
:10638000743CF212709AE4B5464BB55F5DB5685E39
:10639000B57662B57763B54868E4B54949B5476FE6
:1063A000B54470B54C74B56E7AB57A7FB57B4EE561
:1063B0004B454A601DE54B2401F54B5002054A450B
:1063C0004A700FC20D20540A20550712607DD25327
:1063D000D24D02634CD546B2C20D757500740712DA
:1063E0007031D24280A4154980B3155F809FD56873
:1063F0009FC264809B1576809A15778099157B8063
:10640000AED5489575450330180302584C808A155F
:1064100047808DD5448DD2468089D54C89126AF744
:10642000E48083D56E83C2A70263A9157A0263ACA8
:10643000E51DA2E3304E0292A330510292A23050E9
:106440000292A122C2B6204702D2B612644F327520
:10645000C800C2ADC2AC75CBFF75CA9875CDFF75CB
:10646000CC98759853C298C299D2ACC2BC75C83446
:106470007599062275C800C2ACC2AD75980075CC7E
:106480002B75CDEBD2AD75C8042275C800C2ACC265
:10649000AD759800E58A242BF5CC540F658C24EB60
:1064A000F5CDD2AD75C80422C2A8C2AAC289C28BDA
:1064B000C2ACC2A9C2AB758F01120759D2181260C3
:1064C00094126073E4F53B784FF2787275F010F235
:1064D000D5F0FCC254C255C256753DFF753FFF75DD
:1064E0001D04C23F1289BA754800C242D24C756B76
:1064F00000C233C21AC21BD246C247754410E4F52B
:1065000040F541F542F534F5361220A4751E0075AC
:106510001F80E4F546F54EF54DF554F555F53EC2B0
:1065200025C226C227C20374377855F27856F2780E
:1065300057F27858F2D221754503754701C2137896
:106540001AE47A07F208DAFCC2147550FF789CA6A8
:1065500050C215C20C757603755F1E756000C25B74
:10656000C211C212C20DC20EC20FC257C258755D0F
:1065700000755C0075F006782AE4F208D5F0FB7926
:1065800043E4F309F37945F309F37847E4F212158C
:10659000E87549FAB2B57532FF7533FFD25C75679D
:1065A000007829740AF2126ED2C264756801C208BA
:1065B000C209C205C206C207D2A0756E00756F007F
:1065C00075700078A274FAF2E478ADF278AEF278E1
:1065D000AFF278A3743CF2C268C267C263757500FB
:1065E00012700DC269D26AC26BD26D1215A9757A8A
:1065F00000757B00758901758A3E758C5DC2B9D2C4
:10660000A9D28CD2B612644FD2AFD293C2B4D2B256
:10661000B2B522C218754F0375F003128908D5F080
:10662000FAC257C258122624754F0375F003128917
:1066300008D5F0FAC257C2581224B3C2AF12157F60
:1066400002000020071020060820090A200802C3C3
:1066500022126A85D322126BE3D322C26D75F00039
:10666000C0F0127756D0F0500343F008E5F0223026
:106670006714203E2278AFE2306506C265600214DE
:10668000F224FA50092230680E78AFE27009E574FE
:10669000540170031200E422C268C267E478AFF2CA
:1066A00022C2AF7549FAB2B5128920B2B51289205B
:1066B000B2B5D2A07581D375D0001264A8125E2F36
:1066C000125CFD126113121EC87549FA120E921265
:1066D0006643754F031227A21227B81200F1C2AF0A
:1066E000751880751904751A84120BD4D219300CE0
:1066F0000F120CAE125D4A125D9D125C4A125E4E84
:10670000C26CD2B7D2AFC218C219000000D2B7D241
:10671000AFC218C21900000020B70912892020B7A3
:1067200003021EE2300C32120CAE12666FE5725498
:1067300020601178A2E2D5E00A126992125BE1783A
:10674000A274FAF2E57560021575300C0C125D4A00
:10675000125D9D125C4A125E4EE5606003D5600ECC
:1067600012700612289E125B99125BD0800CD2A385
:10677000C24EC2A1D250D2A4C24FE55F7003125CD8
:10678000E7C251D2A1C250125E39C257C258D25389
:10679000785BE2600D24FD4009756D0212299512A7
:1067A0006643785CE2600D24FD4009756D03122993
:1067B00095126643E5715440600620A8031287DFF6
:1067C000122334204908204805204A02801E302D1B
:1067D0000D740712707A5006125E2F0267E41236AB
:1067E000511266437829E215E0F270087829741492
:1067F000F202670D0267440074A212688CE8126806
:10680000C7E91268C71268FE2274A212688CE812E7
:1068100068C7E71268C709D582F81268FE2274A219
:1068200012688CE81268C774A312688C1268E7F7C4
:1068300009D582041268FE22C296D297000000C2D7
:106840009780E974A212688CE81268C71268502217
:1068500074A312688C1268E7F91268FE2274A27A97
:1068600008C296000000C297335005D296026872A3
:10687000C296D297000000C297DAEDD29600D29766
:10688000000000309604C297C322D3227A08D29621
:10689000D29700000000000000000000000000008F
:1068A0000000C296000000C297335005D2960268DD
:1068B000B3C296D297000000C297DAEDD29600D20A
:1068C00097000000C297227A08335005D2960268DA
:1068D000D3C296D297000000C297DAEDD29600D2CA
:1068E00097000000C297227A08D296C29700000053
:1068F00000D297C3309601B333DAF0C29722C29622
:10690000000000D297000000D29622781079B2C021
:106910008275820512681ED08278B2B6870E08B6DC
:10692000E00A08B6330608B6A902C322D3221269C8
:106930000B40012278AC76000876000876000876D5
:106940000108760178AA760008760078AEE6543F12
:10695000F6780079AAC082758207126809D082127F
:106960008908781479AAC082758207126809D082D2
:1069700012890878B276870876E00876330876A917
:10698000781079B2C082758204126809D0821289A7
:106990000822780279ACC08275820512681ED08206
:1069A0002278B0E603C4540775F018A4C0E078AEAE
:1069B000E6C4540375F00AA4F5F0E6540F25F0D0B0
:1069C000F025F075F03CA4C0F0C0E078ADE6C4540A
:1069D0000775F00AA4F5F0E6540F25F0D0F025F085
:1069E000F5F0D0E03400C5F022206956205D21C0CA
:1069F000D0C0E0E8C0E0C0F0E54C700375690075F8
:106A00004C02D260126AB5D0F0D0E0F8D0E0D0D01D
:106A1000C28932205D29C0D0C0E0E8C0E0C0F0E506
:106A20004C7003756900754C02A2B2B39260126C8F
:106A30003B308502D205D0F0D0E0F8D0E0D0D0C213
:106A40008B32C2A8C289322069C9205D26C0D0C05D
:106A5000E0E8C0E0C0F0E54C7003756900754C02D9
:106A6000C260126AB5308502D205D0F0D0E0F8D00D
:106A7000E0D0D0C28B32C2A8C2AAC293C2B4C0E0D6
:106A8000128908D0E0C269C293C2B4C289C28BD253
:106A9000B2D2B3C25D754C00756900C205C2B8D2EE
:106AA00088D2A8C2BAD28AD2AA22C269C2A8C2AA6D
:106AB000C289C28B22E5697007A260925E026AD821
:106AC0001475F00884B409047569002250FA243A58
:106AD000F8E2A260925F33F2056922E56975F00879
:106AE00084243AF8E5F0600E7408C395F0F5F0E2FE
:106AF000C333D5F0FBF222205D22EFC0E0E569242C
:106B0000EE50131569126ADB1569126B2D400712DE
:106B10006B68D25D8003126A85D0E0FF22EF75F0CA
:106B2000088405F0243AF8E233D5F0FC22E569C385
:106B300013C0E0500104C0E07F00C0E0126B1DD024
:106B4000E05002B25E0FD5E0F1D0E0D0F0205E164A
:106B5000AFF0C0E0126B1DD0E05002B25F0FD5E085
:106B6000F1305F02C322D32279307A0AE4F309DAE2
:106B7000FCAF691F79397A04126B1DE392E413F3B9
:106B8000DA0E540FF37A0419C3E9943050028019D5
:106B9000DFE6126B1DE392E413F3DA05540FF38082
:106BA00008C2E413DAFB540FF3E569F56A24D75001
:106BB00003756A2822754732126A76304C05C24C3A
:106BC00012027AE5476008305DF1126AAAC3221208
:106BD0006AAAD322C2A8C2AAC293C2B4C0E01289D0
:106BE00008D0E0D269C293C2B4C289C28BD2B2D2F9
:106BF000B3C25D754C00756900C205C2BAD28AD2B3
:106C0000AA22754732126BD4304C05C24C12027A5C
:106C1000E547600C305DF1E5697005126AAAC32290
:106C2000126AAAD322C330E001B330E101B330E2EB
:106C300001B330E301B330E401B322E56975F00537
:106C400084C0E024EED0E040552430F8E2A2609207
:106C5000E503F2E569700BE2541FB40B407569055A
:106C6000803B0569E5F0B40434E2126C25502F54E2
:106C70000FF218E2540FB40F24D3E894307830F2B6
:106C80000404C082F58275F00B08E265F0F5F0D5DA
:106C900082F7D082540F7006D25D75690022126BA4
:106CA000E322010000000000000000000A000000D4
:106CB00000000000000004060000000000000000CA
:106CC000080E0300000000000000000107020000A1
:106CD00000000000000A0608010000000000000497
:106CE00002040F0000000000000806090809000067
:106CF00000000000010E050F0500000000000A0C56
:106D00000A090B0300000000040E0B00040502003A
:106D10000000080E06070804070100000001050A2C
:106D2000040D080E75F00A79BA770009D5F0FA78E3
:106D300030E2FA60430824F25007EA24F328F87A94
:106D40000DE2540FF26029EA1475F00AA424A2F5AA
:106D5000827400346CF58379C37E007B0AE493F57A
:106D6000F0E2A42E2775F01084FEA7F0A319DBED46
:106D700008DACE756A28C322D322094300A0095439
:106D8000009F0966009E0977009D0989009C099B68
:106D9000009B09AD009A09BF009909D2009809E447
:106DA000009709F700960A0A00950A1D00940A3018
:106DB00000930A4300920A5700910A6B00900A7FE1
:106DC000008F0A93008E0AA7008D0ABB008C0AD19F
:106DD000008B0AE7008A0AFE00890B1400880B2B3F
:106DE00000870B4300860B5C00850B7500840B8EBF
:106DF00000830BA700820BC100810BDB00800BF628
:106E0000007F0C10007E0C2B007D0C47007C0C6476
:106E1000007B0C81007A0C9E00790CBB00780CDBA7
:106E200000770CFB00760D1B00750D3B00740D5BAD
:106E300000730D7D00720D9F00710DC200700DE496
:106E4000006F0E07006E0E2C006D0E51006C0E765A
:106E5000006B0E9B006A0EC100690EE900680F11FD
:106E600000670F3900660F6100650F8900640FB37A
:106E700000630FDE00621009006110340060105FD3
:106E8000005F7F42906D7AE493A3F5F0E493A3C38F
:106E9000958BE5F0958D5015A3A3DFEBE58224FFDC
:106EA000F582E58334FFF583E49314800BA3E49328
:106EB000BF4205906D7A8010C0E0E58224F9F5822A
:106EC000E58334FFF583D0E022900063E0A28733AE
:106ED000F0229000647400F09000637455F090000C
:106EE0006574FFF09000677405F09000667412F00E
:106EF000D28122D286A2A4C0D0D2A475F000D5F04F
:106F0000FDD5F0FDC28E53890F438910758B007536
:106F10008D00C28FC2AFC2A4D28E208603308FFAFA
:106F2000C28E308F06758BFF758DFFD2AFD0D09299
:106F3000A422F024FE4005308102C2812290006725
:106F4000E0D5E0EE7442F0126EF3D281E58B249925
:106F5000E58D34F24014E58B24E1E58D34F3400EE9
:106F6000E58B24E0E58D34FC40087415800674112F
:106F700080027412FE900066E06E6015EEF0E5711E
:106F80005404700DC2AF7518C07519008E1A120B1B
:106F9000D422126EC9603B046038900065E020E0A6
:106FA00010D2E0F0900064E070047405F022E4F088
:106FB00022900064E0602E14F0702AE57154027093
:106FC00024C2AF7518C0751900751A14120BD402BB
:106FD0006FE5900065E030E00DC2E0F0900064E005
:106FE00070CC743CF022900064E060F914F070F50D
:106FF000E571540270EFC2AF7518C0751900751AAB
:1070000013120BD480DF126F3D126F92229002E7B1
:1070100075F008E4F0A3D5F0FB9002EF75F008746A
:10702000FFF0A3D5F0FB22C0E012707AD0E0B3509D
:107030002CC0E024F8D0E04022C082C083F5F024C8
:10704000EFF582E43402F583E0C5F024E7F582E44D
:107050003402F583E5F0F0D083D082D322C0E0245F
:10706000F8D0E04013C082C08324E7F582E4340204
:10707000F583E4F0D083D082C322C0E024F8D0E0CE
:107080004016C082C08324E7F582E43402F583E031
:10709000D083D0826002D322C322C082C0839002F8
:1070A000E775F008E06003B4FF09A3D5F0F6D083DC
:1070B000D0822220E70414F080F03066ED14F0B4A2
:1070C00080E8E4F080E4B44008740012707A027141
:1070D00058B44107740112707A807DB4420774027B
:1070E00012707A8073B44307740312707A8069B4A3
:1070F0004407740412707A805FB45407A2717272EC
:10710000B38055B45506A271B072804CB45606A235
:1071100072B0718043B45706A2718272803AB4583B
:1071200007A26F7270B38030B45906A26FB070803E
:1071300027B45A06A270B06F801EB45B06A26F829D
:10714000708015C0E024DED0E040132324C6C0E0E8
:1071500074003471C0E022C3740122D380FAE4C306
:1071600022A23EB380F2D24DA26380EC80F0A20D49
:1071700080E6A20F80E2A26B80DE80DF80E0A20EBC
:1071800080D6A26480D2E56F457060CB80CD12625C
:10719000FA80C5A2567255B380BEA255822880B827
:1071A000A255B02880B2A25680AEC3306709203EF7
:1071B0000678AFE27001D3809FA262B3809AC3E5E4
:1071C000766001D380928099809C809A8098809686
:1071D0008094809280908094809480968098809A09
:1071E000809A809A809C809E80A480A780AC80B08A
:1071F00080B480B680C380C68010801A8027802E1D
:10720000803D804C805B80638018C3203E05E5771D
:107210006001D3027158C3303E05E5776001D302A7
:10722000715802715EA26D027158C3027158E57205
:10723000541070F6303EF3740512707A027158E5FE
:1072400072541070E5303EE2740612707A02715882
:10725000E572541070D4303ED1740712707A027106
:1072600058E57A600302715B027157E57B60F902B1
:10727000715B12736C300C19C0E0C082C08374045F
:10728000120188D083D082D0E040030272A702723C
:1072900091E538B40D0A302302802CD223D3801517
:1072A0001270C66022800EE538B40D06202303025A
:1072B00072C7C223C34009C229A229B392A580077D
:1072C000D229A229B392A5300C19C0E0C082C08394
:1072D0007405120188D083D082D0E040030272F995
:1072E0000272E3E539B40D0A302402802CD224D393
:1072F00080151270C66022800EE539B40D06202478
:1073000003027319C224C34009C22AA22AB392A657
:107310008007D22AA22AB392A6300C19C0E0C082FC
:10732000C083740B120188D083D082D0E040030266
:10733000734B027335E53AB40D0A300202802CD249
:1073400002D380151270C66022800EE53AB40D0695
:1073500020020302736BC202C34009C204A204B339
:1073600092808007D204A204B3928022B21030101F
:107370006CE57254106003303E27E57354047007C7
:10738000740512707A4040E5735401700774061258
:10739000707A4015E57354027007740712707A40D2
:1073A00017C263754E000273DDE54EB401028024FE
:1073B000754E01754D40801CE54EB4020280157576
:1073C0004E02754DA0800DE54EB403028006754E49
:1073D00003754DF0E54D23F54DA2E0926322C229DD
:1073E000A229B392A522D229A229B392A522B22919
:1073F000A229B392A522F5F00303543FB40258E545
:107400003864086005E538B40D4AE5F089F0C0F04D
:10741000300C19C0E0C082C0837404120188D0838C
:10742000D082D0E0400302743B02742CD0F0A9F06B
:107430005403B4020D1273DE027520D0F0A9F002DD
:107440007520B401061273E6027520B403061273A8
:10745000EE02752002751EB40362E539640860050A
:10746000E539B40DEFE5F089F0C0F0300C19C0E05B
:10747000C082C0837405120188D083D082D0E040DE
:107480000302749A027487D0F0A9F05403B4021175
:10749000C22AA22AB392A6027520D0F0A9F00275E2
:1074A00020B4010AD22AA22AB392A6027520B403FC
:1074B00009B22AA22AB392A680668062B4045FE56C
:1074C0003A64086005E53AB40D54E5F089F0C0F07F
:1074D000300C19C0E0C082C083740B120188D083C5
:1074E000D082D0E040030274FE0274ECD0F0A9F028
:1074F0005403B4020FC204A204B392808022D0F0DD
:10750000A9F0801CB40109D204A204B392808010B7
:10751000B40309B204A204B3928080048000D32291
:10752000C322C0E07417306221B53807C229A229EE
:10753000B392A5B53907C22AA22AB392A6B53A07D3
:10754000C204A204B39280D0E022B53807D229A2A7
:1075500029B392A5B53907D22AA22AB392A6B53A81
:1075600007D204A204B39280D0E022C0E012774395
:10757000D0E04023302C03203E1D20561AC0E012DC
:107580006099126087D0E020380BC2AF1288B175C5
:107590001810120BD4D32220380BC2AF1288B17549
:1075A0001820120BD4C322D20F757A10C2AF7518EF
:1075B000C0751900751A01120BD4302826205529E0
:1075C00020360DC2AF754AFF754BF8D2AF12607D01
:1075D000784DE2F546E5745410600312445C789DE2
:1075E00076FF222034031276B122C256C2552054AF
:1075F00009C0E0126073D0E0D253543F44C0C2AF20
:10760000F51A7519087518C0020BD4D256C2552048
:107610005409C0E0126073D0E0D253543F4480C29A
:10762000AFF51A7519087518C0020BD4D255C25699
:10763000205409C0E0126073D0E0D253543F44405C
:10764000C2AFF51A7519087518C0020BD4D255C20D
:1076500056205409C0E0126087D0E0D253543F4412
:1076600000C2AFF51A7519087518C0020BD430178F
:107670000122C0E074108004C0E0741178C6760A5C
:107680000875F00A84F608A6F0753C03D0E078A9E6
:10769000F2087405F2D21722C20F75460074071261
:1076A000705DC2AF7518C0751900751A02120BD43F
:1076B000227575007405127031C2AF7518507519B6
:1076C0000F751AFF120BD422C23ED26DC2AF7518CD
:1076D0006075190F751AFF120BD47577031244B336
:1076E000C24022D23EC26DC2AF75187075190F75B7
:1076F0001AFF120BD475770322C0E0126113D0E099
:10770000543F4400C2AFF51A75190B7518C0120B1F
:10771000D422786CF208F212286EC2AF7518C075C8
:107720001900751A50120BD422400C305408C25460
:10773000205503126073222054FC12609912608756
:10774000D25422127ABD400D127EBB40081282B97B
:1077500040031286BA22127AC8400D127EC6400833
:107760001282C440031286C522A290301E01B37853
:1077700055E233F222106A03027B66301808C378A0
:1077800055E4F2027AD6E57354106003303EEF7888
:1077900055E260EF046003027B6420210320254F43
:1077A000D225300C19C0E0C082C083740012018859
:1077B000D083D082D0E04003027B640277BE785150
:1077C000E224A4401CC082C083907A05E225E00434
:1077D00093F5F0E225E093D083D082C0F0C0E0E2E0
:1077E00022E2C2AF751890751909F51A120BD4026E
:1077F0007B64125E391200D7027B6474011275A794
:10780000027B64740112756B40E8027B641276C8D7
:10781000027B64D2647568050277E2C0E0740112ED
:107820007031D0E00277E2203E0320350CC0E074D6
:1078300004127031D0E00277E2027B64743D027979
:10784000080277E2C0E0E57454047005D0E00277E6
:10785000E2D0E0027B64C0E0D37401127729D0E06B
:107860000277E20277E20277E2740012766E027B20
:1078700064741012766E027B64741112766E027B51
:1078800064742012766E027B647401F974AAF87530
:107890002F0075308C7531F112060B78AAE612763E
:1078A0006E027B647401F974AAF8752F0075308C30
:1078B0007531F112060B78AAE6127678027B6430F5
:1078C000681E78AEE2601978AFF27401543F4480CC
:1078D000C2AF7518C0751909F51A120BD40277F2E8
:1078E000027B643068FAE478AFF27401543F44409C
:1078F000C2AF7518C0751909F51A120BD40277F2C8
:1079000074011276F90277F2203E061276E30277CE
:10791000F21276C80277F2E57154106007E412772C
:10792000120277F2027B64E5715410600874FF1252
:1079300077120277F2027B6474011275EA027B64AB
:10794000740112764D027B64740112762C027B6402
:10795000740112760B027B64740012703174011290
:1079600089540277F2740012705D74011289650205
:1079700077F2740012707A40EC0279587402127037
:107980003174011289760277F2740212705D74010B
:107990001289870277F2740212707A40EC02797CC5
:1079A000740312703174011289980277F274031211
:1079B000705D74011289A90277F2740312707A4023
:1079C000EC0279A0303E03027911027B64203EFA7A
:1079D00002790B7400440112889B0277F274400212
:1079E00079D574800279D574C00279D574004401C8
:1079F0001288850277F274400279EE74800279EE83
:107A000074C00279EE7B6477FB7803780D77E277B8
:107A1000E277E27813781B7827783C77E278417830
:107A200044785677E277E277E277E277E277E277B7
:107A3000E277E277E277E277E277E277E277E2777E
:107A4000E277E277E277E277E277E277E277E2776E
:107A5000E277E277E277E277E277E277E277E2775E
:107A6000E277E277E277E277E278637866786978BE
:107A70007178797881788978A478BF78E37900790A
:107A80000879177927793879407948795079587980
:107A9000657972797C7989799679A079AD79BA77A7
:107AA000E279C479CD77E277E277E277E279D37948
:107AB000DD79E279E779EC79F679FB7A007851E2C1
:107AC000B40B03A22522C322203E097851E2B40D53
:107AD00003A22522C322202106202503027B64C2A3
:107AE00025300C19C0E0C082C0837400120188D018
:107AF00083D082D0E04003027B64027AFD7851E2B9
:107B000060DAB40106127698027B64B40203027B49
:107B100064B403051276E3804BB40908203E363086
:107B200035338040B40A02743DB40D0BE57454043F
:107B30007032740D027B55B40E0BC3740112772999
:107B4000740E027B55C0E024CED0E05008C0E02483
:107B5000B0D0E0500FC2AF7518A0751909F51A1210
:107B60000BD48000D26A22A291301F01B37856E272
:107B700033F222106A03027F64301808C37856E497
:107B8000F2027ED4E57354206003303EEF7856E273
:107B900060EF046003027F6220210320264FD2267B
:107BA000300C19C0E0C082C0837401120188D083F8
:107BB000D082D0E04003027F62027BBC7852E22494
:107BC000A4401CC082C083907E03E225E00493F5AC
:107BD000F0E225E093D083D082C0F0C0E0E222E260
:107BE000C2AF75189075190AF51A120BD4027F628C
:107BF000125E391200D7027F6274021275A7027FEB
:107C000062740212756B40E8027F621276C8027FCE
:107C100062D264756805027BE0C0E07401127031C5
:107C2000D0E0027BE0203E0320350CC0E07404125B
:107C30007031D0E0027BE0027F62743D027D06027B
:107C40007BE0C0E0E57454047005D0E0027BE0D036
:107C5000E0027F62C0E0D37402127729D0E0027B99
:107C6000E0027BE0027BE0740012766E027F6274B9
:107C70001012766E027F62741112766E027F627449
:107C80002012766E027F627401F974AAF8752F00D3
:107C900075308C7531F512060B78AAE612766E02F5
:107CA0007F627401F974AAF8752F0075308C7531F4
:107CB000F512060B78AAE6127678027F6230681E0B
:107CC00078AEE2601978AFF27402543F4480C2AFDC
:107CD0007518C0751909F51A120BD4027BF0027FD2
:107CE000623068FAE478AFF27402543F4440C2AFA5
:107CF0007518C0751909F51A120BD4027BF07402BD
:107D00001276F9027BF0203E061276E3027BF01237
:107D100076C8027BF0E57154106007E41277120216
:107D20007BF0027F62E5715410600874FF127712D5
:107D3000027BF0027F6274021275EA027F627402B3
:107D400012764D027F62740212762C027F627402F8
:107D500012760B027F627400127031740212895421
:107D6000027BF0740012705D7402128965027BF070
:107D7000740012707A40EC027D56740212703174F5
:107D800002128976027BF0740212705D740212890D
:107D900087027BF0740212707A40EC027D7A7403E1
:107DA0001270317402128998027BF0740312705DB4
:107DB00074021289A9027BF0740312707A40EC02FB
:107DC0007D9E303E03027D0F027F62203EFA027DDF
:107DD000097400440212889B027BF07440027DD338
:107DE0007480027DD374C0027DD374004402128873
:107DF00085027BF07440027DEC7480027DEC74C0DF
:107E0000027DEC7F627BF97C017C0B7BE07BE07B7D
:107E1000E07C117C197C257C3A7BE07C3F7C427CB9
:107E2000547BE07BE07BE07BE07BE07BE07BE07B06
:107E3000E07BE07BE07BE07BE07BE07BE07BE07B6A
:107E4000E07BE07BE07BE07BE07BE07BE07BE07B5A
:107E5000E07BE07BE07BE07BE07BE07BE07BE07B4A
:107E6000E07BE07BE07BE07C617C647C677C6F7C1A
:107E7000777C7F7C877CA27CBD7CE17CFE7D067D5F
:107E8000157D257D367D3E7D467D4E7D567D637D0F
:107E9000707D7A7D877D947D9E7DAB7DB87BE07D16
:107EA000C27DCB7BE07BE07BE07BE07DD17DDB7D39
:107EB000E07DE57DEA7DF47DF97DFE7852E2B40B4C
:107EC00003A22622C322203E097852E2B40D03A267
:107ED0002622C322202106202603027F62C22630EA
:107EE0000C19C0E0C082C0837401120188D083D015
:107EF00082D0E04003027F62027EFB7852E260DAC9
:107F0000B40106127698027F62B40203027F62B463
:107F100003051276E3804BB40908203E3630353332
:107F20008040B40A02743DB40D0BE5745404703201
:107F3000740D027F53B40E0BC37402127729740EB2
:107F4000027F53C0E024CED0E05008C0E024B0D07F
:107F5000E0500FC2AF7518A075190AF51A120BD4AC
:107F60008000D26A22A292302001B37857E233F225
:107F700022106A03028362301808C37857E4F202C1
:107F800082D2E57354406003303EEF7857E260EFF1
:107F900004600302836020210320274FD227300C86
:107FA00019C0E0C082C0837402120188D083D082DD
:107FB000D0E04003028360027FBA7853E224A440F9
:107FC0001CC082C083908201E225E00493F5F0E2B8
:107FD00025E093D083D082C0F0C0E0E222E2C2AFBD
:107FE00075189075190CF51A120BD4028360125E85
:107FF000391200D702836074031275A7028360747C
:108000000312756B40E80283601276C8028360D267
:1080100064756805027FDEC0E07401127031D0E043
:10802000027FDE203E0320350CC0E0740412703164
:10803000D0E0027FDE028360743D028104027FDEB5
:10804000C0E0E57454047005D0E0027FDED0E002A9
:108050008360C0E0D37403127729D0E0027FDE0290
:108060007FDE027FDE740012766E0283607410126F
:10807000766E028360741112766E02836074201231
:10808000766E0283607401F974AAF8752F0075305A
:108090008C7531F712060B78AAE612766E028360B1
:1080A0007401F974AAF8752F0075308C7531F712C8
:1080B000060B78AAE612767802836030681E78AEE6
:1080C000E2601978AFF27403543F4480C2AF751870
:1080D000C0751909F51A120BD4027FEE02836030C5
:1080E00068FAE478AFF27403543F4440C2AF7518A5
:1080F000C0751909F51A120BD4027FEE74031276BB
:10810000F9027FEE203E061276E3027FEE1276C879
:10811000027FEEE57154106007E4127712027FEEE1
:10812000028360E5715410600874FF127712027FB9
:10813000EE02836074031275EA02836074031276A0
:108140004D028360740312762C02836074031276EE
:108150000B02836074001270317403128954027F21
:10816000EE740012705D7403128965027FEE740074
:1081700012707A40EC02815474021270317403124E
:108180008976027FEE740212705D74031289870291
:108190007FEE740212707A40EC02817874031270E0
:1081A000317403128998027FEE740312705D7403B8
:1081B0001289A9027FEE740312707A40EC02819C4E
:1081C000303E0302810D028360203EFA0281077473
:1081D00000440312889B027FEE74400281D17480B8
:1081E0000281D174C00281D17400440312888502D7
:1081F0007FEE74400281EA74800281EA74C00281D9
:10820000EA83607FF77FFF80097FDE7FDE7FDE808D
:108210000F8017802380387FDE803D804080527F32
:10822000DE7FDE7FDE7FDE7FDE7FDE7FDE7FDE7F66
:10823000DE7FDE7FDE7FDE7FDE7FDE7FDE7FDE7F56
:10824000DE7FDE7FDE7FDE7FDE7FDE7FDE7FDE7F46
:10825000DE7FDE7FDE7FDE7FDE7FDE7FDE7FDE7F36
:10826000DE7FDE7FDE805F80628065806D8075806E
:108270007D808580A080BB80DF80FC8104811381AC
:10828000238134813C8144814C81548161816E81A0
:108290007881858192819C81A981B67FDE81C081B0
:1082A000C97FDE7FDE7FDE7FDE81CF81D981DE8107
:1082B000E381E881F281F781FC7853E2B40B03A2F9
:1082C0002722C322203E097853E2B40D03A22722BD
:1082D000C322202106202703028360C227300C1905
:1082E000C0E0C082C0837402120188D083D082D0E3
:1082F000E040030283600282F97853E260DAB4015D
:1083000006127698028360B40203028360B4030508
:108310001276E3804BB40908203E36303533804076
:10832000B40A02743DB40D0BE57454047032740D3C
:10833000028351B40E0BC37403127729740E0283A7
:1083400051C0E024CED0E05008C0E024B0D0E050CE
:108350000FC2AF7518A075190CF51A120BD4800056
:10836000D26A22A285300101B37858E233F222109A
:108370006A03028768301808C37858E4F20286D38B
:10838000E57354806003303EEF7858E260EF04609C
:108390000302876620210320034FD203300C19C04B
:1083A000E0C082C083740A120188D083D082D0E0FA
:1083B00040030287660283B87854E224A4401CC0BC
:1083C00082C083908602E225E00493F5F0E225E086
:1083D00093D083D082C0F0C0E0E222E2C2AF751831
:1083E0009075190DF51A120BD4028766125E3912B8
:1083F00000D702876674041275A702876674041298
:10840000756B40E80287661276C8028766D264758B
:1084100068050283DCC0E07401127031D0E0028391
:10842000DC203E0320350CC0E07404127031D0E033
:108430000283DC028766743D02850502876602833B
:10844000DCC0E0E57454047005D0E00283DCD0E0C9
:10845000028766C0E0D37404127729D0E00283DC7F
:108460000283DC0283DC740012766E02876674106D
:1084700012766E028766741112766E028766742019
:1084800012766E0287667401F974AAF8752F00756A
:10849000308C7531F312060B78AAE612766E0287DD
:1084A000667401F974AAF8752F0075308C7531F374
:1084B00012060B78AAE612767802876630681E7874
:1084C000AEE2601978AFF27404543F4480C2AF75D5
:1084D00018C0751909F51A120BD40283EC028766CD
:1084E0003068FAE478AFF27404543F4440C2AF7588
:1084F00018C0751909F51A120BD40283EC74041212
:1085000076F90283EC203E061276E30283EC1276C3
:10851000C80283ECE57154106007E41277120283FD
:10852000EC028766E5715410600874FF127712023E
:1085300083EC02876674041275EA0287667404127B
:10854000764D028766740412762C028766740412D4
:10855000760B02876674001270317404128954021B
:1085600083EC740012705D74041289650283EC74EC
:108570000012707A40EC0285557402127031740456
:108580001289760283EC740212705D74041289877A
:108590000283EC740212707A40EC02857974031243
:1085A000703174041289980283EC740312705D7444
:1085B000041289A90283EC740312707A40EC0285DC
:1085C0009D303E0302850E028766203EFA02850832
:1085D0007400440412889B0283EC74400285D274B8
:1085E000800285D274C00285D2740044041288854A
:1085F0000283EC74400285EB74800285EB74C00248
:1086000085EB876683F583FD840783DC83DC83DC6D
:10861000840D84158421843683DC843B8441845317
:1086200083DC83DC83DC83DC83DC83DC83DC83DC52
:1086300083DC83DC83DC83DC83DC83DC83DC83DC42
:1086400083DC83DC83DC83DC83DC83DC83DC83DC32
:1086500083DC83DC83DC83DC83DC83DC83DC83DC22
:1086600083DC83DC83DC846084638466846E84764C
:10867000847E848684A184BC84E084FD8505851481
:1086800085248535853D8545854D85558562856F74
:10869000857985868593859D85AA85B783DC85C187
:1086A00085CA83DC83DC83DC83DC85D085DA85DFE7
:1086B00085E485E985F385F885FD7854E2B40B03FC
:1086C000A20322C322203E097854E2B40D03A20380
:1086D00022C322202106200303028766C203300C36
:1086E00019C0E0C082C083740A120188D083D0828E
:1086F000D0E040030287660286FA7854E260DAB47A
:108700000106127698028766B40203028766B403F4
:10871000051276E38050B40908203E3B303538809E
:1087200045B40A02743DB40C02803BB40D0BE574F1
:1087300054047032740D028757B40E0BC3740412C4
:108740007729740E028757C0E024CED0E05008C0CD
:10875000E024B0D0E0500FC2AF7518A075190DF528
:108760001A120BD48000D26A22E5715440601AE5D7
:108770007254027006127769127775E572540470AC
:1087800006127B67127B73800C1277691277751261
:108790007B67127B73127F65127F71128363128372
:1087A0006FC22120420122C242C2AF7518C07519A2
:1087B00000751A54120BD422E8C0E07851E2640329
:1087C00060187852E2640360117853E26403600A2F
:1087D0007854E264036003C38001D3D0E0F822E45C
:1087E000A22892E0A22992E1A22A92E2A20492E3B4
:1087F000F56C756D051227E474035004122970227C
:1088000012294878A3E6C0E0E57254026012D0E075
:10881000C0E0540712883DD0E0C0E0540712883D04
:10882000E57254046014D0E0C0E0C45407128861BB
:10883000D0E0C0E0C45407128861D0E022A2253005
:108840001E01B34007D320E10A028860C320E2037F
:10885000028860301E01B3E494007855F2127775F7
:1088600022A226301F01B34007D320E10A028884E8
:10887000C320E203028884301F01B3E494007856D9
:10888000F2127B7322A2E6926FA2E79270C2AFF55A
:108890001A75190D7518C0120BD422A2E69271A296
:1088A000E79272C2AFF51A75190F7518C0120BD482
:1088B00022B4010775190F751AE122B40207751960
:1088C0000F751AE222B4030775190F751AE322B463
:1088D000040775190F751AE422B4110775190F757D
:1088E0001AD122B4120775190F751AD222B41307C0
:1088F00075190F751AD322B4140775190F751AD488
:108900002275190F751AD422C28E53890F4389100C
:10891000758BD6758D97C28FD28E308FFDC28E2209
:10892000C28E53890F438910758BEB758DCBC28F27
:10893000D28E308FFDC28E22C28E53890F43891092
:10894000E58AC4242BF58B758DEBC28FD28E308FC8
:10895000FDC28E22543F4400C2AFF51A75190A7544
:1089600018C0020BD4543F4480C2AFF51A75190ADF
:108970007518C0020BD4543F4400C2AFF51A7519E4
:108980000C7518C0020BD4543F4440C2AFF51A75A1
:10899000190C7518C0020BD4543F4480C2AFF51AAD
:1089A00075190C7518C0020BD4543F44C0C2AFF502
:1089B0001A75190C7518C0020BD4740112705D740D
:1089C0000412705D1244B322000000000000000099
:1089D0000000000000000000000000000000000097
:1089E0000000000000000000000000000000000087
:1089F0000000000000000000000000000000000077
:108A00000000000000000000000000000000000066
:108A10000000000000000000000000000000000056
:108A20000000000000000000000000000000000046
:108A30000000000000000000000000000000000036
:108A40000000000000000000000000000000000026
:108A50000000000000000000000000000000000016
:108A60000000000000000000000000000000000006
:108A700000000000000000000000000000000000F6
:108A800000000000000000000000000000000000E6
:108A900000000000000000000000000000000000D6
:108AA00000000000000000000000000000000000C6
:108AB00000000000000000000000000000000000B6
:108AC00000000000000000000000000000000000A6
:108AD0000000000000000000000000000000000096
:108AE0000000000000000000000000000000000086
:108AF0000000000000000000000000000000000076
:108B00000000000000000000000000000000000065
:108B10000000000000000000000000000000000055
:108B20000000000000000000000000000000000045
:108B30000000000000000000000000000000000035
:108B40000000000000000000000000000000000025
:108B50000000000000000000000000000000000015
:108B60000000000000000000000000000000000005
:108B700000000000000000000000000000000000F5
:108B800000000000000000000000000000000000E5
:108B900000000000000000000000000000000000D5
:108BA00000000000000000000000000000000000C5
:108BB00000000000000000000000000000000000B5
:108BC0000000000000000000000000000000505203
:108BD000343032207665722E3133322E332E3020EF
:108BE0004864773A482030352D30312D30362030EA
:108BF000303A353420200043524300000000005139
:00000001FF
:0300000306028072
